:10000000029EC60298EB12B90A00220289BE12288B
:100010001CFF90FDCB126F581270887403F07D5056
:1000200002929302A83690FEAE126FAB90FEAE1213
:100030006F58F912A7E290FEAE126F58126F917DC1
:1000400009129293A212E433FF22FF02964F7865C1
:100050000622FF02941512281CFF90FDD7126F583C
:100060001270887414F07D6002929302A2D090FD09
:100070006212889DA3EDF012AD9BC22FE490FA941A
:10008000F0A3F090FD65E0547FFF90FA94E0FCA3AC
:10009000E0FDC39F7480F8EC648098507C90FD6212
:1000A000128805128817FF12883C90FDDEEDF09053
:1000B000FD65E0547F90FDDFF0128347EF7002FF93
:1000C0002290FA92E0C394105034E490FA96F0A390
:1000D000F0128852501812881D1288CA601090FAC7
:1000E00097E004F070EB90FA96E004F080E3128859
:1000F00052400D1288841288371288B68002D22F9F
:1001000012883C7D051296FE90FA95E004F0700688
:1001100090FA94E004F002008390FD65E090FF8087
:10012000F090FD66E090FF81F090FD62128805126C
:10013000884CC003C002C00190FD6212880512887D
:1001400017FD90FD917401F0A374FFF0A37482F089
:10015000D001D002D00312B30912883C7D0A129656
:10016000FE12863A90FD6712889D90FD6212880506
:10017000128817FF12883C12AFA790FD67E0FBA31F
:10018000E0FAA3E0F8AC0212883A7F141288CC603F
:1001900004C2308002D23090FD66E0540FFFC39459
:1001A00007400BEF440890FA91F0C230801A90FD9E
:1001B00066E0540FFF90FA91E0FEEFD39E4002807C
:1001C00002AF0690FA91EFF090FD65E0FFC3941046
:1001D0004017EF94105003E004F090FD65E0448078
:1001E000F090FA92F0C230800A302F0790FA92E035
:1001F0004480F0A230E433FF2290FC25EFF022FF90
:10020000000200B9FFEA0D0A496E46696C653A20A2
:1002100070726F6A6563742E6865780D0A4F757425
:10022000446174653A20323031312F31312F303111
:100230000D0A4F757446696C653A206B6C39372E20
:100240006865780000000000000000000000000069
:10025000000000000000000000000000000000009E
:10026000000000000000000000000000000000008E
:10027000000000000000000000000000000000344A
:1002800090FC9AEB125C61E490FCA1F07B0190FC85
:10029000AB04F0A374FFF07480125EA774FFF074D7
:1002A0009E125EA774FFF0A374CBF0A3EBF0A374CF
:1002B000FFF0A374CEF0A3EBF0A374FFF0A374EDF2
:1002C000F090FC9A125B9FEA494B7002FF2290FE6D
:1002D00041E0640260030203CC90FC9A125B9F121F
:1002E0005E0630E04A125BDBF8AC02AD03A3125BA2
:1002F0009F125E0C125C02125B9C125D29703090A2
:10030000FC9A125B9F125E0630E124125D0490FCA1
:100310009D125BED125EAEC003C002C001125BEA2B
:10032000125DB8D001D002D003125E0C125C0290B4
:10033000FC9A125B9F121AAF7003021A3E90FC9A4D
:10034000125B9F90FCA3E0125BCA541FC39407503A
:1003500003021A3E125CF390FCA0E030E02D90FC0A
:10036000A3E0FF7E002406125C09D3942D50030203
:100370001A3E125DEA54BF125E8A125B9F125BD274
:10038000C3942D500280337F2D802F90FCA3E0FF7B
:100390002406125E74125B9F125C0DD3941E5003F0
:1003A000021A3E125DEA548F125E8A125B9F125B44
:1003B000D2C3941E500280027F1E90FCA3E024064C
:1003C000F582E433F583125BFE021A3E125B9C1247
:1003D0005F35D3940140037F002290005A122835E4
:1003E000707490005B122835706C90005C12283598
:1003F000706490005D12283564FD705A125CA21280
:100400005C83C39412EE64809480504A125B9CEF2C
:10041000245AFFE43EFE8F82F58312283590FCA615
:10042000F090FE43E0246CFD125C2F125EC28F82BE
:100430008E8312289690FCA6E0FF90FE43E0246C89
:10044000FD125C2F8D82F583EF122896125C93705B
:10045000AE125CC680A990FC9A125B9F125E0630B9
:10046000E012125BDBF8AC02AD03A3125B9F125EDD
:100470000C125C02125E13600302054A90FC9A1291
:100480005B9F125E1AFF125B9C125E1A4F4421FFA3
:1004900090FCAB125B9F125E20125B9F125E28FFE6
:1004A000125B9C125E284F4408FF90FCAB125B9FCE
:1004B000125D32125B9F125E2EFF125B9C125E2E4B
:1004C0004FFF90FCAB125B9F125D71125B9C900022
:1004D0006C122835600302061390006D12283560F7
:1004E0000302061390006E12283560030206139073
:1004F000006F12283564FD600302061390FC9A1207
:100500005B9F90006C12283560030205E990006D36
:1005100012283560030205E990006E122835600349
:100520000205E990006F12283564FD701A9000757D
:10053000122835FF125B9C900075122835D39F500E
:10054000030206130205E60205E990FC9A125B9F7E
:10055000125E1AFF125B9C125E1A5F4421FF90FC30
:10056000AB125B9F125E20125B9F125E28FF125B34
:100570009C125E285F4408FF90FCAB125B9F125DEB
:1005800032125B9F125E2EFF125B9C125E2E5FFF8B
:1005900090FCAB125B9F125D71125B9C125EB560AA
:1005A00072125EBBFF606C90FC9A125B9F125EB58C
:1005B0006037125EBBFE6031EFC39E5002802A900E
:1005C000FC9A125B9F125EBBFF125B9C125EBB6FBC
:1005D000704190FC9A125B9F125EB5FF125B9C12F9
:1005E0005EB5C39F502DE9800690FC9D125BED2403
:1005F00036F9E43AFAC003C002C001125BEA2436BD
:10060000125DBAD001D002D0037E007F481227F6D7
:10061000125C0290FC9A125B9F125E1AFF90FCAB78
:10062000125B9F12281CFE6F7021125D78125B9F77
:10063000125E28B5071590FCAB125B9F900002126A
:100640005D7B125B9F125E2E6F6003125C0290FC5A
:100650009A125B9F900023EE12289690FCAB125BDF
:100660009F125D78125B9F900024EF12289690FCF9
:10067000AB125B9F900002125D7B125B9F90002586
:10068000EF125C9A125C83125E98501390FC9A12DF
:100690005B9F125BD2125C8D70EA125CC680E51221
:1006A0005DCA125B9F90007FEF1228967E007F1E2E
:1006B0007D0090FCAB125B9F1231387E007F2D7D58
:1006C0000090FCAE125B9F125F3B90FCB1125B9FEF
:1006D0001231387E007F1F7D0090FCB4125B9F12A8
:1006E0005F3B90FCB7125B9F123138E490FCA6F0A0
:1006F00090FCA8F090FCA7F090FCA9F0A3F090FC6F
:100700009A125B9F125D29600302087D125B9C12A6
:100710005F35600302087D90FC9A125B9F125E06B3
:1007200030E203021AA9125F45FF54C0440190FC55
:10073000A6F06F6003125C02125E137040125D59E6
:1007400090FC9A125B9F121AC0605090FC9A125B48
:100750009F125BC5125C69801F125CB950E2125E89
:10076000CF501590FC9A125B9F8E82125BCCFF904B
:10077000FCAB125B9F125C73125CF380DC90FC9A02
:10078000125B9F900084122835541F640660031288
:100790005C02125CCE125B9F12B472125D5990FC27
:1007A0009A125B9F121AD3603590FC9A125B9F12CB
:1007B0005BC5125C698022125CB950E2125ED750B0
:1007C0001890FC9A125B9F8E82125BCCFF90FCAE5D
:1007D000125B9F90FCA8125C76125CF380D990FCAF
:1007E0009A125B9F121AE6604590FC9A125B9F1268
:1007F0005BC5125C69125CF3125D16125BCCFF9054
:10080000FCB1125B9F125E20125B9F125D13125BA4
:10081000CCFF90FCB1125B9F125D32125B9F125DA8
:1008200013125BCCFF90FCB1125B9F125D7190FCC8
:100830009A125B9F121AAF603590FC9A125B9F125E
:100840005BC5125C698022125CB95022125EDF50D7
:100850001890FC9A125B9F8E82125BCCFF90FCB4C6
:10086000125B9F90FCA9125C76125CF380D9125C3B
:100870000290FE41E060030216ED0216E2125B9C5C
:10088000125D2960030216A6125C9E125C83C3945B
:1008900080EE648094805012125B9C7480125DE044
:1008A000125C8C70E6125CC680E190FE40E0604A0B
:1008B000125BEA2400125D0690FC9A125B9F900086
:1008C0007E7401125BFF125B9C125F4554C04401B1
:1008D00090FCA6125CCD125B9F12B472125C459024
:1008E000FCAE125B9F121B43125B9F12B49890FEEA
:1008F00041E060030216ED0216E290FC9A125B9F43
:10090000125E06FE30E203021AA9EE30E124125D07
:100910000490FC9D125BED125EAEC003C002C001EC
:10092000125BEA125DB8D001D002D003125E0C1245
:100930005C02125B9C900083125D7B125B9F125FD6
:1009400045FE5F54F0444190FCA6F06E6003125CDB
:1009500002125E136003020A23125D5990FC9A1280
:100960005B9F121AC0603290FC9A125B9F125BC5AB
:10097000125C69801F125CB950E2125ECF50159074
:10098000FC9A125B9F8E82125BCCFF90FCAB125BD9
:100990009F125C73125CF380DC125DC3125B9C12CD
:1009A0001AF77003020ADC125B9C90FCA2125BC86F
:1009B00090FCA4125C6C125CB2125D83D39F50DC7D
:1009C000E4125CA290FCA7E0FF125C1B125CFA50E0
:1009D00025125B9C90FCA2E0125BCA547FFF90FC46
:1009E000AB125B9F125C0D547F6F600A125C9370B8
:1009F000D3125CC680CE90FCA7125F4B125CE8401D
:100A00001CEF941E5017125B9C90FCA2E0125BCA74
:100A1000FF90FCAB125B9F90FCA7125BF5125EE7A8
:100A20000209B9125D5990FC9A125B9F90FCA3E0F9
:100A300090FE26F07D40121B8B7003020ADC90FCB6
:100A40009A125B9F125BC5125C69020AD6125EEFB6
:100A500050D4125DC3125B9C121AF76079125B9C32
:100A600090FCA2125BC8125F558038125D83FED3E2
:100A70009F503590FC9A125B9F90FCA3E0125BCADA
:100A8000FF547FFD125B9C8E82125BCCFE547FB5BF
:100A90000511125ECF500CEE4FFF90FCAB125B9F26
:100AA000125C73125CB280C390FCA7E0602224FF4A
:100AB000FFE434FFFE90FCAB125B9F125BD290FC14
:100AC0009A125B9F90FCA3E0125BCA6F6087800064
:100AD000125C02020A55125CF3020A4D90FE41E0DC
:100AE000FF64016008EF64036003020DEB125D59BF
:100AF00090FC9A125B9F121AD3603590FC9A125B9D
:100B00009F125BC5125C698022125CB950E2125ED2
:100B1000D7501890FC9A125B9F8E82125BCCFF908C
:100B2000FCAE125B9F90FCA8125C76125CF380D93D
:100B3000125DC3125B9C121B0A7003020CDC125B79
:100B40009C90FCA2125BC8125CA9125D83D39F50DB
:100B5000E2E4125CA290FCA8125CE04003020C7A72
:100B6000125B9C90FCA2E0125BCAFF5478FE90FEE0
:100B700040BE0805747FF080037478F090FE40E07A
:100B80005FFF90FCAE125B9F125F5F8C8312283573
:100B9000FE90FE40E05E6F6003020C6C125B9C9066
:100BA000FCA2E0125BCA5407FFEE5407FED39F403D
:100BB00004AF068000125B9C90FCA2E0125BCA545A
:100BC000784FFF90FCAE125B9F125C1BF5828C830A
:100BD000EF122896125DB1FFE433FE125B9C125BAC
:100BE000D290FCAE125B9FED2401FDE43C125EC18D
:100BF0004F8D828C83122896125C83F5828E83122D
:100C000028355478FDBD082B90FCAE125B9F125D19
:100C1000A5E92FF9EA3EFAC003C002C00112281C60
:100C2000125B91125C0D4FD001D002D003122884C8
:100C3000020C7A125DD5125B9C125BD290FCAE1254
:100C40005B9F90FE43E02402FD125C2F125EC1FE0A
:100C5000D39F4004AF068009125DD5125B9C125BE6
:100C6000D290FCAE125B9F125D45800E90FE43E079
:100C70002403F0125C2FF0020B5590FCA8125F4B7E
:100C8000125CE84051EF942D504C125B9C90FCA2FA
:100C9000125BC8FE90FCAE125B9F125F69EE1228D9
:100CA00096EF2401FFE433FE125B9C125BD2ED242D
:100CB00001125D93125B9F125D45125DD5125B9C24
:100CC000125BD2125D8D125B9F125D4590FCA8E015
:100CD0002403F0125C02125EE7020B4A90FC9A12A7
:100CE0005B9F121AE6603FE004F090FC9A125B9F53
:100CF000125D13125BCCFF90FCB1125B9F125E2061
:100D0000125B9F125D13125BCCFF90FCB1125B9FD4
:100D1000125D32125B9F125D13125BCCFF90FCB12F
:100D2000125B9F125D71125B9C121B6970030210B3
:100D300037E004F0125B9C90FCA2125BC8FE90FCB2
:100D4000B1125B9F12281C6E6003125C027E00EFE2
:100D50002401FDEE125B9A125C0DFD90FCB1125B5A
:100D60009F125E346003125C02125DA5125B9C123E
:100D70005BD290FCB1125B9F125E3C6003125C027E
:100D800090FCB1125B9FC003C002C00112281CFF7F
:100D9000125B9C90FCA2E0125BCA4FD001D002D043
:100DA00003125F73125BED2401F9E43AFAC003C049
:100DB00002C001125DAD125B98125C0D4FD001D0E4
:100DC00002D003125F73125BED2402F9E43AFAC019
:100DD00003C002C00112281C125B91125C0D4FD09F
:100DE00001D002D003122884021037125D5990FC02
:100DF0009A125B9F90FCA3E090FE26F07D20121BD0
:100E00008B7003020F7390FC9A125B9F125BC512EA
:100E10005C69125CF3125EEF50D4125DC3125B9CEE
:100E2000121B0A7003020F69125B9C90FCA2125BFA
:100E3000C8125CA9125D83FED39F50E1125B9C8EA9
:100E400082125BCCFF5478FE90FE40BE0805747F92
:100E5000F080037478F090FC9A125B9F90FCA3E002
:100E6000125BCAFE90FE40E0FD5EFCED5F6C60032D
:100E7000020F32125ED74003020F32EE5407FF1208
:100E80005B9C90FCA2E0125BCA5407FEC39F500417
:100E9000AF06801090FC9A125B9F90FCA3E0125B5F
:100EA000CA5407FF125B9C90FCA2E0FE125BCA547E
:100EB000784FFF90FCAE125B9F125F69EF1228968D
:100EC00090FCA3E02401FDE433FC90FC9A125B9FAC
:100ED000125C0DFFEE2401125B98125C0D5FFF9017
:100EE000FCA8E0FE2401125D93125B9F125D458E0B
:100EF00082125BCC54786408700A125B75125C0D28
:100F00005FFF801E125B75125C0DFEC39F5004AF25
:100F100006800F90FCA3E02402125D69125B9F1211
:100F20005BD2125D8D125B9F125D4590FCA8E024A0
:100F300003F090FCA8E0FF602724FDFFE434FFFEEF
:100F400090FCAE125B9F125E44547FFF90FC9A129D
:100F50005B9F90FCA3E0125BCA547F6F600580002A
:100F6000125C02125EE7020E3490FCA3E02403F050
:100F7000020E1590FC9A125B9F90FE267484F07D01
:100F80008012A34790FCA3EFF07003021037125BAE
:100F90009C121B697003021037E004F0A3E004F018
:100FA00090FC9A125B9F90FCA3E0125BCAFF125B5D
:100FB0009C90FCA2E0125BCA5FFF90FCB1125B9FA9
:100FC000EF125D60125B9F125BD2125DB1125B98F3
:100FD000125C0D90FCB1125B64125C0D5FFF90FC23
:100FE000B1125B9F900002125D35125B9F125BC5D0
:100FF000FE90FCB1125B9F12281C6E6003125C0213
:101000007E00EF2401125E76125B9F125C0DFD9054
:10101000FCB1125B9F125E346003125C02125DA58C
:1010200090FC9A125B9F125BD290FCB1125B9F12F4
:101030005E3C6003125C02125E1360030212869033
:10104000FC9A125B9F121B58603590FC9A125B9FB2
:10105000125BC5125C698022125CB95022125EFBE1
:10106000501890FC9A125B9F8E82125BCCFF90FC12
:10107000B4125B9F90FCA9125C76125CF380D912CB
:101080005B9C121B7A7003021451125B9C90FCA2B1
:10109000125BC8125CA9E4125CA2125C1490FCA45E
:1010A000125E4B400302145190FCA9E0FFC3ED9F78
:1010B000EC6480984003021260125C8364064E6008
:1010C00018EF64084E6012EF64094E600CEF640A7A
:1010D0004E6006EF640B4E7079125C142FFFEE3CED
:1010E000FE125B9C125BD290FCB4125B9F125C0DF3
:1010F000FED39F4004AF06800A125C24FE125B9C64
:10110000125BD290FCB4125B9F125C1BF5828C8345
:101110001228356F6003125C0290FCA2E07E002D65
:10112000FFEE3CFE125B9C125BD290FCB4125B9F04
:10113000125C0DFED39F4004AF06800A125C24FEB1
:10114000125B9C125BD290FCB4125B9F125F5F0239
:10115000125B125C83C39405EE64809480503F90D0
:10116000FCA0E020E10302127B125D9BFDEC3E122D
:101170005B9B125C0DFD90FCB4125B9F125E446D94
:101180006003125C02125C142FFFEE3CFE125B9CAB
:10119000125BD290FCB4125B9F8D8202125B125CD8
:1011A00083C3940DEE64809480504E125D9BFDECE1
:1011B0003E125B9B125C0DFD90FCB4125B9F125EB5
:1011C000446D6003125C0290FE42E0FEA3E029F948
:1011D000EA3EFAC003C002C00112281CFF90FCA224
:1011E000125DFD125C2F125B9B125C0D4FD001D083
:1011F00002D00312288402127B125F20125B9C1221
:101200005BD2125E5BFFE433FE90FCB4125B9F90F6
:10121000000D122835FDC4135407FBED541F2BFDA0
:10122000E433FC125D4D5053125C142FFFEE3CFE74
:10123000125B9C125BD290FCB4125B9F125C0D6F30
:101240006003125C02125C142FFFEE3CFE125B9CEA
:10125000125BD290FCB4125B9F8D82125D47801BA3
:10126000125EFB5016125C24FE125B9C125BD29045
:10127000FCB4125B9F90FCA9125BF5125C937003A7
:10128000125CC602109A90FC9A125B9F121B587057
:1012900003021451125B9C121B7A70030214511248
:1012A0005B9C90FCA2125BC8125F5590FC9A125B8B
:1012B0009F125BC5125C69125CB2A3E004F0E412F9
:1012C0005CA290FCA3125C1790FCA5125E4B40033D
:1012D00002143090FCA2E0F9FF7E00ED2FFFEE3CFF
:1012E000FE90FCA4E0FDD3EF9D74806E9840030255
:1012F0001430125EFB4003021425125C8364064E18
:101300006018EF64084E6012EF64094E600CEF64E1
:101310000A4E6006EF640B4E7032E9125C28FE1232
:101320005B9C125BD2125DFA125C2FFC90FC9A124D
:101330005B9F125C0DFEC39F5005AF060213F612B1
:101340005C24FE125B9C125BD20213F6125C83C318
:101350009405EE64809480502690FCA0E030E10C6F
:10136000125D9BFFEC3EFE90FC9D800A90FCA31258
:101370005C27FE90FC9A125B9F125BD20213F6125E
:101380005C83C3940DEE648094805024125D9BFFB7
:10139000EC3EFE125B9C125BD2125DFA90FE42E0C4
:1013A0003CFC90FC9A125B9F125C0D5FFF0213F6EF
:1013B000125F20125B9C125BD2125E5BFFE433FE75
:1013C000C006C00790FCA3E0240D125D69125B9F6C
:1013D000125BD2125E5BFDE433FCD007D006125DD7
:1013E0004D500990FCA3125C27FE8007125C24FE7E
:1013F000125B9C125BD290FCB4125B9F90FCA91212
:101400005C7690FCA3125C172FFFEE3CFE90FC9ADA
:10141000125B9F125BD290FCB4125B9F125C0D6F4B
:101420006003125C02125C937003125CC60212C26B
:1014300090FCA3E024FFFFE434FFFE90FC9A125BD3
:101440009F125E44541FFF90FCA9E06F6003125C82
:101450000290FCB4125B9F7403125E83125B9F9038
:101460000001740C122896E4125D7290FCA0E0FF5B
:1014700030E21590FCB4125B9F90000374101228A8
:1014800096900004E4122896125EDF50037405F073
:1014900090FCA9E0C394074058EF30E02890FCB4DA
:1014A000125B9F125EC9D3942D4046125E6554BFF5
:1014B000125E7E125B9F125EC9FFC3942D500280A4
:1014C0002A7F2D802690FCB4125B9F125EC9D394B4
:1014D0001E401E125E65548F125E7E125B9F125E6E
:1014E000C9FFC3941E500280027F1E900006125B4B
:1014F000FE125E1360030215E6125D5990FC9A120B
:101500005B9F121B1D604190FC9A125B9F125BC592
:10151000125C69125CF3E0125BCAB405DF125CB9BD
:1015200050DA90FCAAE0C39403501890FC9A125B26
:101530009F8E82125BCCFF90FCB7125B9F90FCAA3F
:10154000125C76125CF380D5125DC3125B9C121B99
:101550003070030216ED125B9C90FCA2125BC81265
:101560005CA9125BC8B405E37E00EF2401125C099C
:10157000FD90FCB7125B9F125E346003125C021296
:101580005DA5125B9C125BD290FCB7125B9F125E52
:101590003C6003125C02125F03125BED2401F9E46C
:1015A0003AFAC003C002C001125DAD125B98125C32
:1015B0000D4FD001D002D003125F05125BED240263
:1015C000F9E43AFAC003C002C00112281C125B9170
:1015D000125C0D4FD001D002D00312288490FCAAD7
:1015E0007403F002154B125D5990FC9A125B9F1226
:1015F0001B1D70030216ED90FC9A125B9F125BC5D7
:10160000125C69125CF3E0125BCA640560030216A7
:10161000ED125DC3125B9C121B3070030216ED12BB
:101620005B9C90FCA2125BC8125CA9E0125BCA64CE
:101630000560030216ED90FCB7125B9F7405125D06
:1016400060125B9F125BD2125DB1125B98125C0D4F
:1016500090FCB7125B64125C0D5FFF90FCB7125BED
:101660009F125D7190FCAA7403F090FCA3E0FF242C
:1016700001125E74125B9F125C0DFD90FCB7125B51
:101680009F125E346003125C02125DA590FC9A12F8
:101690005B9F125BD290FCB7125B9F125E3C604D69
:1016A000125C020216ED125BEA2400125D0690FC49
:1016B0009A125B9F90007E7401125BFF90FCA674EF
:1016C00041125CCD125B9F12B472125C4590FCAE6D
:1016D000125B9F121B43125B9F12B49890FE41E075
:1016E000700B125BEA125F0C440412288490FC9A7F
:1016F000125B9F125D296003021A3E90FCA7E0C3B3
:1017000094015009125CCE125B9F12B47290FE419C
:10171000E0B4042990FD297401F0A374FCF0A374D3
:10172000A8F090FCB1E0F9A3E0FAA3E090FD2C1240
:101730005C6090FCAE125B9F12AE8A801590FCA894
:10174000E0C39403500C125C4590FCAE125B9F12F8
:10175000AE50125EDF501790FDBF7401F0A374FC11
:10176000F0A374A9F090FCB4125B9F12B498E41239
:101770005CA290FCA7E0FF125C1B125CFA50169072
:10178000FCAB125B9F125C0D20E70A125C9370E2C7
:10179000125CC680DD90FCA7125CE0400E90FCABB2
:1017A000125B9F12281C4480122884E490FCA3F052
:1017B000125BB0125D1D7402122884125BB0FF042C
:1017C000F0125D22740312288490FCA8E0FF90FCC4
:1017D000A7E02FFF90FCA9E02FFFA3E060047E0F9D
:1017E00080027E0BEF2EFF125BB07C0029F9EC3AF1
:1017F000FAEF12288490FCA8E01475F01E841228D9
:1018000062125CF390FCA6E0125BAFFE04F0EE12F5
:101810005C3C90FCA7E04440125BAFFE04F0EE128B
:101820005C3CE4125CA290FCA7E0FF125C1B125C23
:10183000FA501690FCAB125B9F125BA8125C36123A
:101840005C9370E2125CC680DD90FCA8E0D3941E2D
:10185000406F125BB0125D1D743E122884E4125C6E
:10186000A2125C83C3941EEE64809480501A90FC94
:10187000AE125B9F8F828E83125BAC125C36125C61
:101880009370DE125CC680D990FCA8E024E2FFE4ED
:1018900034FFFE90FCAE125BED241EF9E43AFAC070
:1018A00003C00290FCAEA3E0FAA3E0F8AC02AD03E3
:1018B000D002D0031227F690FCA8E024E2F0021830
:1018C0004990FCA8E04420125BAF125C36E4125C45
:1018D000A290FCA8E0FF125C1B125CFA501690FC70
:1018E000AE125B9F125BA8125C36125C9370E21220
:1018F0005CC680DD125BB0125D1D7483125F7312D3
:101900005B9F12281C125BAF125C3690FCB1125B1D
:101910009F900001125BACFE04F0EE125C3C90FC68
:10192000B1125B9F900002125BACFE04F0EE125C01
:101930003C90FCA9E04460125BAFFE04F0EE125C48
:101940003CE4125CA290FCA9E0FF125C1B125CFA62
:10195000501690FCB4125B9F125BA8125C36125CAE
:101960009370E2125CC680DD90FCAAE0FFD3940085
:101970004035EF44E0125BAF125C36125BB0125D93
:101980001D125F03125B9F900001125BACFE04F01E
:10199000EE125C3C90FCB7125B9F900002125BACB5
:1019A000FE04F0EE125C3CE4125CA290FCA7E0FFA7
:1019B000125C1B125CFA505C90FCA3E0C3946E5066
:1019C0005390FCAB125B9F125C0D547FFF6401606F
:1019D00038EFC3943C5032EF75F012A4242BF97405
:1019E0004D35F0FA7BFFC003C002C001125BB07E30
:1019F0000029F9EE125DBCD001D002D0037F121293
:101A000027F690FCA3E02412F0125C937003125CA2
:101A1000C60219AB90FCA3E0FFFDC374809DFDE4FA
:101A20009400FCC004C005125BEA125EAEEF7C00BD
:101A300029F9EC3AFA7D00D007D006123138125C51
:101A40009D125C83125E98501390FC9A125B9F1259
:101A50005BD2125C8D70EA125CC680E5125DCA1220
:101A60005B9F90007FEF122896125D29703B90FCDF
:101A70009A125B9F9000FEE4125C9A125C83125EE5
:101A8000985019125BEA125EAEE92FF9EA3EFA129B
:101A9000281C125C8C70E4125CC680DF125DCA12D6
:101AA0005B9F9000FFEF12289690FCA1E0FF229030
:101AB000FE267484F07D6012A34790FCA3EFF02211
:101AC00090FCA3E090FE26F07D4012A34790FCA37B
:101AD000EFF02290FCA3E090FE26F07D2012A347B9
:101AE00090FCA3EFF02290FE267484F07D8012A378
:101AF0004790FCA3EFF02290FCA2E090FE26F07D40
:101B00004012A34790FCA2EFF02290FCA2E090FECE
:101B100026F07D2012A34790FCA2EFF02290FCA3B8
:101B2000E090FE26F07DE012A34790FCA3EFF022A8
:101B300090FCA2E090FE26F07DE012A34790FCA26C
:101B4000EFF02212AE5090FDBF7401F0A374FCF0D0
:101B5000A374A9F090FCB42290FE267484F07D60FA
:101B600012A34790FCA3EFF02290FE267484F07D30
:101B70008012A34790FCA2EFF02290FE267484F01E
:101B80007D6012A34790FCA2EFF02212A34790FCC5
:101B9000A3EFF02290FE101272A9900006122D03FE
:101BA00090FE131272A990FE1312723B4A4B7003FF
:101BB0000227251271FE12281CD394015003021C27
:101BC000CD127254C003C002C0011271FE127243E2
:101BD000D001D002D00312A259EF60111271FE128F
:101BE00072F520E50812734F7003021CCD1271FECE
:101BF000127254C003C002C0011271FE127243D0AF
:101C000001D002D00312B658127238240412723175
:101C100054FD1271FB127254C003C002C001127154
:101C2000FE127243D001D002D00312B5931271FE9E
:101C3000127254C003C002C0011271FE127243D06E
:101C400001D002D00312B6381271E61272A01273DC
:101C50004F30E7291271FE127254C003C002C00156
:101C60001271FE127243D001D002D00312A259EFBA
:101C700090FE106005127201800D021CBF1271FEF1
:101C800012734FFF30E60474028039EF90FE10307B
:101C9000E52D127201127254C003C002C00112710C
:101CA000FE127243D001D002D00312B55112723825
:101CB000240412723144041271FB1273388005122D
:101CC000720174011228841271FE1273DC1271FE0B
:101CD00012281CB40700400302223B901CE2F828A3
:101CE0002873021CF7021E2302200C02202402206B
:101CF0005B0220790221B5127254C003C002C001F8
:101D00001271FE127243D001D002D00312B6389085
:101D1000FE1312720112281C704B1273F290FE1007
:101D200030E40C12723B24051272314410800A1206
:101D3000723B240512723154EF12288490FE131264
:101D400072011273F290FE1030E50D12723B240501
:101D50001272314420021DE712723B2405127231C7
:101D600054DF021DE7127238240512723154EF124B
:101D7000288454DF1271FB127254C003C002C001E8
:101D80001271FE127243D001D002D00312B551126B
:101D900071FE127254C003C002C0011271FE1272B1
:101DA00043D001D002D00312AC18EF700C1272387D
:101DB00024051272314410802E1271FE127254C02A
:101DC00003C002C0011271FE12724390FD7C1273B7
:101DD0002CD001D002D0031297A5EF700D127238EB
:101DE000240512723144100228841272382405121C
:101DF000723154EF1228841271FE127254C003C063
:101E000002C0011271FE127243D001D002D003123F
:101E1000B6381271E612727B7D0412871F1271FEB2
:101E20000222DA1271FE127254C003C002C0011203
:101E300071FE127243D001D002D00312A25990FC5D
:101E40002CEFF070030222E71271FE1272F530E5FA
:101E5000030222E71272CB940AEE9400500302228E
:101E6000E790FC2CE0B402181273E39464E5F0945C
:101E70000050030222E7E92404127231547F800AE1
:101E8000127238240412723144801228841271FEB6
:101E9000127419FF12741F127426EF601B1271FE68
:101EA0001273E39419E5F0940050030222E7E92449
:101EB000051272314440800A1272382405127231C0
:101EC00054BF1228841271FE1272A012741F129B4A
:101ED000F5EF90FE10605512723B240412723144EB
:101EE0000112288412741F90FE267484F07D601203
:101EF000A3477E00749C2FF9EE34FAFA90FDE37448
:101F0000011272AA1271FE12727B12B04A1271FE95
:101F100012727B7D0212A78D1271FE12727BC003BA
:101F2000127281D003E4FD12A42D800D12723B24A5
:101F30000412723154FE1228841271FE1272F530AE
:101F4000E01A127254C003C002C0011271FE127274
:101F500043D001D002D00312B5D5801B1271FE12FE
:101F60007254C003C002C0011271FE127243D0014C
:101F7000D002D00312B6781271FE12727BE94A4B7E
:101F800060381271FE12727B12734F30E02C1271A6
:101F9000FE12725412B883EF600D1271FE1272F5C8
:101FA00030E6047F0180027F00EF44041273961232
:101FB0007201120280EF604F803D1271FE12725466
:101FC00012B883EF600D1271FE1272F530E6047FD5
:101FD0000180027F001271FE127419FE90FC25E050
:101FE000B506047E0280027E00EE4F1273961272D6
:101FF00001120280EF601090FE1312723B24011256
:10200000723144401228841271FE80131271FE1244
:1020100072CB940AEE940050030222E71272A0746D
:10202000030222DC90FE1312720112281CD39403C7
:1020300050030222E71271FE127254C003C002C0A4
:10204000011271FE127243D001D002D00312B59377
:102050001271FE1272A074040222DC1271FE12725E
:10206000CB9408EE940050030222E712724B12AE9A
:10207000C41271FE74050222DC1271FE1272CB943E
:1020800096EE9400500C90FE131272011272F5300D
:10209000E17B1271FE1272A01272F520E22B127116
:1020A000FE127254C003C002C0011271FE127243CC
:1020B000D001D002D00312B551127238240412722A
:1020C00031440412288412B4BE1271FE127254C03C
:1020D00003C002C0011271FE127243D001D002D0BF
:1020E00003120026EF70261271FE127254C003C054
:1020F00002C0011271FE127243D001D002D003124D
:10210000B6381271E61272A074060222DC1271FE59
:10211000127254C003C002C0011271FE127243D089
:1021200001D002D00312A259EF6401703E1271FE79
:102130001272F520E72990FE10A3A3E0127254C09A
:1021400003C002C0011271FE127243D001D002D04E
:102150000312B6381271E61272A0740112288412AA
:10216000723824041272314480800A1272382404B6
:10217000127231547F12288490FE1312720112726F
:10218000F520E1030222E71271FE127254C003C06F
:1021900002C0011271FE127243D001D002D00312AC
:1021A000B551127238240412723144041271FB12B8
:1021B00073380222DC1271FE1272CB94FAEE940094
:1021C00050030222E712724BC003C002C001127119
:1021D000FE127243D001D002D00312B551127238F0
:1021E0002404127231440412288412B4BE1271FE07
:1021F000127254C003C002C0011271FE127243D0A9
:1022000001D002D003120026EF60081271FE7403A1
:102210001228841271FE127254C003C002C001124F
:1022200071FE127243D001D002D00312B63812727E
:1022300038240412723154FB0222DC1271FE127235
:1022400054C003C002C0011271FE127243D001D00B
:1022500002D003120026EF60201271FE127254C0E9
:1022600003C002C0011271FE127243D001D002D02D
:102270000312A259EF640160681271FE127254C019
:1022800003C002C0011271FE127243D001D002D00D
:102290000312B658127238240412723154FD1271AE
:1022A000FB127254C003C002C0011271FE127243CD
:1022B000D001D002D00312B5931271FE127254C035
:1022C00003C002C0011271FE127243D001D002D0CD
:1022D0000312B6381271E61272A0740112288480BB
:1022E000061271FE1247B51271FE12281CFF640C13
:1022F000601EEFD394024018EF64066013EF640D84
:10230000600790FA92E020E70790FA91E030E30A44
:10231000E924041272314410800A12723824041223
:10232000723154EF1228841271FE12727B129FDAFE
:1023300040030225801271FE12727B127329A3E4FE
:10234000F0A37413F012ACE090FF80E0122D8C2308
:102350008F0023CF0323DA0523E206240407242C6D
:1023600008244B0924690C248B0D24BA1024C211B3
:1023700024D71224E51325001424E515251116256C
:102380001E17252B18253E19254D1A000025809073
:10239000FF92E0FDB405047E0180027E0090FC2BDC
:1023A000EEF090FC29740112740DEDB4050890FC58
:1023B000327405F0801390FF92E0B40F0890FC3265
:1023C000740FF08004127321F012736702242490BA
:1023D000FC29741BF0E4A302246012722544080255
:1023E000257D78267CFC1272727E007F031227F610
:1023F0001271FE12727B12730A12B07F12722544A0
:102400001002257D90FC297410F0A314F090FF9227
:10241000E0B405047F05800590FC2DE0FF90FC32C0
:10242000EF127266127222444002257D90FC2974DC
:1024300012F0740F1273CCB405047F05800590FC74
:102440002DE0FF12720A444002257D74131273C6F8
:10245000B405047F05800590FC2DE0FF90FC32EF71
:10246000F0127225444002257D90FC297415F0A3DA
:102470007406F090FF92E0B405047F05800590FC9F
:102480002DE0FF12720A444002257D74161273C6B5
:10249000FFB405047E05800590FC2DE0FE90FC3223
:1024A000EEF01272254440122884EF6405600302A6
:1024B0002580127225448002257D12722544200257
:1024C000257D7407127319F012726E7E007F081258
:1024D0007222444002257D7408127319F01272258D
:1024E000444002257D90FC297409F0741112731F79
:1024F000F012726E7E007F10127222444002257D1F
:1025000078437CFC1272727E007F0E1227F6022541
:102510008074141272B2127225444002257D740D2B
:102520001272B2127225444002257D90FC29740E6D
:10253000F0A3740912732012720E4440803F90FC85
:1025400029740F1272B51272254440803090FC2914
:102550007417F0A37403F090FC3274051272C190EA
:10256000FF84E0600790FC2DE0FF80027F0090FC7C
:1025700034EFF012722544401228844480122884DB
:102580001271FE12736130E127E924021272315494
:10259000FD122884E490FC32F01271FE12727B90DE
:1025A000FD45741AF0A37401F0A312728C0226DFA9
:1025B0001271FE12736130E218E924021271F212F4
:1025C000727BC00390FD45741B127286D0030226F5
:1025D000DF1271FE12736130E31DE92402127231C1
:1025E00054F71271FB12727BC00390FD4574061202
:1025F0007286D0030226DF1271FE12736130E42965
:10260000E9240212723154EF1271FB12727B1273C1
:102610000A12B07F1271FE12727BC00390FD4574E6
:102620000C127286D0030226DF1271FE1273613023
:10263000E61CE9240212723154BF1271FB12727B44
:1026400090FC2BE0FD1273AC12728C0227121271F7
:10265000FE12736120E703022725E924021272317A
:10266000547F12288490FC32E064057042A3E06439
:102670000470151271FE12727B1272DAA3E4F0A3D9
:10268000F0A3F0127FB6800A90FC33E0700FA374C1
:10269000FFF01271FE12727B7D0202A78D1271FE95
:1026A00012727B1272DAA3E4F0A3F0A30227219046
:1026B000FC33E06404702C1271FE12727B1272DA29
:1026C000127355F0127FB61271FE12727B7D0212E8
:1026D000A78D1271FE12727BC003127281D003E4C7
:1026E000FD802F90FC33E0702CA37404F01271FE77
:1026F00012727B7D0412871F1271FE12727B7D02A3
:1027000012A78D1271FE12727BC003127281D00368
:10271000E4FD02A42D1271FE12727B1272DA1273A2
:1027200055F0127FB622E709F608DFFA8046E7097E
:10273000F208DFFA803E88828C83E709F0A3DFFA93
:102740008032E309F608DFFA8078E309F208DFFA5D
:10275000807088828C83E309F0A3DFFA8064898229
:102760008A83E0A3F608DFFA805889828A83E0A38F
:10277000F208DFFA804C80D280FA80C680D480696B
:1027800080F28033801080A680EA809A80A880DA68
:1027900080E280CA803389828A83ECFAE493A3C8FA
:1027A000C582C8CCC583CCF0A3C8C582C8CCC583BC
:1027B000CCDFE9DEE7800D89828A83E493A3F60803
:1027C000DFF9ECFAA9F0EDFB2289828A83ECFAE0CA
:1027D000A3C8C582C8CCC583CCF0A3C8C582C8CC69
:1027E000C583CCDFEADEE880DB89828A83E493A3B9
:1027F000F208DFF980CC88F0EF60010E4E60C388EC
:10280000F0ED2402B4040050B9F582EB2402B404C4
:102810000050AF232345822390277673BB0106899E
:10282000828A83E0225002E722BBFE02E3228982F1
:102830008A83E49322BB010CE58229F582E5833A81
:10284000F583E0225006E92582F8E622BBFE06E980
:102850002582F8E222E58229F582E5833AF583E4D0
:102860009322BB010989828A83F8E028F022500371
:1028700027F722BBFE05F8E328F3228A838982F832
:10288000E4932822BB010689828A83F0225002F752
:1028900022BBFE01F322F8BB010DE58229F582E59A
:1028A000833AF583E8F0225006E92582C8F622BB78
:1028B000FE05E92582C8F222EF8DF0A4A8F0CF8CA6
:1028C000F0A428CE8DF0A42EFE22BC000BBE002961
:1028D000EF8DF084FFADF022E4CCF875F008EF2F17
:1028E000FFEE33FEEC33FCEE9DEC984005FCEE9DD4
:1028F000FE0FD5F0E9E4CEFD22EDF8F5F0EE8420F0
:10290000D21CFEADF075F008EF2FFFED33FD400750
:10291000985006D5F0F222C398FD0FD5F0EA22C2F6
:10292000D5EC30E709B2D5E4C39DFDE49CFCEE3064
:10293000E715B2D5E4C39FFFE49EFE1228CAC3E4A4
:102940009DFDE49CFC80031228CA30D507C3E49F98
:10295000FFE49EFE22C5F0F8A3E028F0C5F0F8E5FC
:1029600082158270021583E038F022A3F8E0C5F0EA
:1029700025F0F0E582158270021583E0C838F0E892
:1029800022BB0110E58229F582E5833AF583E0F563
:10299000F0A3E0225009E92582F886F008E622BB80
:1029A000FE0AE92582F8E2F5F008E222E5832AF53D
:1029B00083E993F5F0A3E99322BB010FF8E582299F
:1029C000F582E5833AF583E802296B5011C5822927
:1029D000F808C5F026C6F5F018C58236C622BBFE3B
:1029E00015C58229F808E2C5F025F0F218E2C58283
:1029F0003582F2E58222E5832AF583E993F5F0A397
:102A0000E993C5F022BB010DC58229C582C5833A71
:102A1000C5830229555011C58229F808E5F026F62C
:102A200018F5F0E58236F622BBFE11C58229F808BA
:102A3000E225F0F5F0F218E23582F222F8E582297B
:102A4000F582E5832AF58374019325F0F5F0E4938C
:102A50003822F8BB0111E58229F582E5833AF58336
:102A6000E8F0E5F0A3F0225009E92582C8F608A6AF
:102A7000F022BBFE09E92582C8F2E5F008F222E85F
:102A80008FF0A4CC8BF0A42CFCE98EF0A42CFC8A53
:102A9000F0EDA42CFCEA8EF0A4CDA8F08BF0A42DD0
:102AA000CC3825F0FDE98FF0A42CCD35F0FCEB8E71
:102AB000F0A4FEA9F0EB8FF0A4CFC5F02ECD39FE27
:102AC000E43CFCEAA42DCE35F0FDE43CFC2275F09C
:102AD00008758200EF2FFFEE33FECD33CDCC33CC23
:102AE000C58233C5829BED9AEC99E58298400CF53E
:102AF00082EE9BFEED9AFDEC99FC0FD5F0D6E4CE6C
:102B0000FBE4CDFAE4CCF9A88222B800C1B900599F
:102B1000BA002DEC8BF084CFCECDFCE5F0CBF9786C
:102B200018EF2FFFEE33FEED33FDEC33FCEB33FB00
:102B300010D703994004EB99FB0FD8E5E4F9FA228A
:102B40007818EF2FFFEE33FEED33FDEC33FCC93385
:102B5000C910D7059BE99A4007EC9BFCE99AF90F4D
:102B6000D8E0E4C9FAE4CCFB2275F010EF2FFFEEB9
:102B700033FEED33FDCC33CCC833C810D7079BEC04
:102B80009AE899400AED9BFDEC9AFCE899F80FD57C
:102B9000F0DAE4CDFBE4CCFAE4C8F922CFF4CFCEEE
:102BA000F4CECDF4CDCCF4CC22E8600FECC313FC12
:102BB000ED13FDEE13FEEF13FFD8F122E86010ECE9
:102BC000A2E713FCED13FDEE13FEEF13FFD8F02286
:102BD000E8600FEFC333FFEE33FEED33FDEC33FC63
:102BE000D8F122BB010789828A830231915005E91D
:102BF000F8022C71BBFE05E9F802319D89828A83B7
:102C00000231A9BB010DE58229F582E5833AF583FE
:102C10000231915007E92582F8022C71BBFE07E9C9
:102C20002582F802319DE58229F582E5833AF58314
:102C30000231A9BB010789828A83022CC65005E9AB
:102C4000F8022CBABBFE05E9F80231E222BB010D05
:102C5000E58229F582E5833AF583022CC65007E91F
:102C60002582F8022CBABBFE07E92582F80231E280
:102C700022E6FC08E6FD08E6FE08E6FF22E6FB0881
:102C8000E6F908E6FA08E6CBF822BB010DE5822951
:102C9000F582E5833AF5830231B95007E92582F8D8
:102CA000022C7DBBFE07E92582F80231C5E58229A9
:102CB000F582E5833AF5830231D2ECF608EDF608A9
:102CC000EEF608EFF622ECF0A3EDF0A3EEF0A3EFA2
:102CD000F022A8828583F0D083D082122CE9122CB6
:102CE000E9122CE9122CE9E473E493A3C583C5F03F
:102CF000C583C8C582C8F0A3C583C5F0C583C8C550
:102D000082C822BB010DE58229F582E5833AF5836D
:102D10000232005007E92582F80231EEBBFE07E9D6
:102D20002582F8023240E58229F582E5833AF5836F
:102D3000023252BB0120E58229F582E5833AF58310
:102D4000D0F0D0E0F8D0E0F9D0E0FAD0E0FBE8C075
:102D5000E0C0F00232375018E92582F8D083D082E3
:102D6000D0E0F9D0E0FAD0E0FBC082C0830231F7B6
:102D7000BBFE18E92582F8D083D082D0E0F9D0E0FC
:102D8000FAD0E0FBC082C08302324922D083D082D5
:102D9000F8E4937012740193700DA3A393F8740177
:102DA00093F5828883E4737402936860EFA3A3A30E
:102DB00080DF8A838982E473E5132582F582E51238
:102DC0003583F583B512048582132210AF06858200
:102DD00013F51222858213F512D2AF22E513258254
:102DE000F582E5123583F58322E3F5F009E208B5B3
:102DF000F06D606B80F3E3F5F009E608B5F0606014
:102E00005E80F387F009E608B5F054605280F487DD
:102E1000F009E208B5F048604680F488828C838728
:102E2000F009E0A3B5F038603680F488828C83879F
:102E3000F009E493A3B5F027602580F388828C83A2
:102E4000E3F5F009E0A3B5F016601480F388828CF6
:102E500083E3F5F009E493A3B5F004600280F20285
:102E60002F14808580E7808E80D2803C8015806C16
:102E7000807E809B80B5808B80A1804F8070803A5F
:102E8000022F2A89828A83ECFAE493F5F0A3C8C55D
:102E900082C8CCC583CCE493A3C8C582C8CCC58303
:102EA000CCB5F070606E80E189828A83E493F5F09E
:102EB000A3E208B5F05E605C80F289828A83E0F567
:102EC000F0A3E608B5F04D604B80F389828A83E079
:102ED000F5F0A3E208B5F03C603A80F389828A837A
:102EE000E493F5F0A3E608B5F02A602880F2805D4F
:102EF00089828A83ECFAE493F5F0A3C8C582C8CC32
:102F0000C583CCE0A3C8C582C8CCC583CCB5F004CA
:102F1000600280E27F00F845F0600EE863F08064B4
:102F200080D395F01F40027F012289828A83ECFAC8
:102F3000E0F5F0A3C8C582C8CCC583CCE0A3C8C562
:102F400082C8CCC583CCB5F0CB60C980E389828AC6
:102F500083ECFAE0F5F0A3C8C582C8CCC583CCE405
:102F600093A3C8C582C8CCC583CCB5F0A760A580A3
:102F7000E288F0ED2402B404005099F582EB2402BB
:102F8000B40400508F2323458223902E6273E3F50F
:102F9000F009E208B5F06BDFF58067E3F5F009E6CC
:102FA00008B5F05EDFF5805A87F009E608B5F05203
:102FB000DFF6804E87F009E208B5F046DFF6804282
:102FC00088828C8387F009E0A3B5F036DFF6803283
:102FD00088828C8387F009E493A3B5F025DFF58020
:102FE0002188828C83E3F5F009E0A3B5F014DFF5C6
:102FF000801088828C83E3F5F009E493A3B5F00296
:10300000DFF40230BD808780E9809080D4803E80EC
:1030100015806E807E809D80B7808D80A3805180DA
:1030200074803C0230C989828A83ECFAE493F5F01B
:10303000A3C8C582C8CCC583CCE493A3C8C582C845
:10304000CCC583CCB5F076DFE3DEE1807089828A7F
:1030500083E493F5F0A3E208B5F062DFF4805E89C3
:10306000828A83E0F5F0A3E608B5F051DFF5804DE4
:1030700089828A83E0F5F0A3E208B5F040DFF580AD
:103080003C89828A83E493F5F0A3E608B5F02EDF4D
:10309000F4802A8002805789828A83ECFAE493F5CF
:1030A000F0A3C8C582C8CCC583CCE0A3C8C582C87C
:1030B000CCC583CCB5F006DFE4DEE280007FFFB54F
:1030C000F0020F2240027F012289828A83ECFAE01B
:1030D000F5F0A3C8C582C8CCC583CCE0A3C8C5821F
:1030E000C8CCC583CCB5F0D5DFE5DEE380CF8982DF
:1030F0008A83ECFAE0F5F0A3C8C582C8CCC583CCBE
:10310000E493A3C8C582C8CCC583CCB5F0AFDFE4D7
:10311000DEE280A988F0EF60010E4E60ABED240284
:10312000B404005098F582EB2402B40400508E23BE
:103130002345822390300573EF4E6012EF60010E3D
:10314000EDBB010B89828A83F0A3DFFCDEFA2289C2
:10315000F05007F709DFFCA9F022BBFEFCF309DF02
:10316000FCA9F022BB010A89828A83F0E5F0A3F072
:10317000225006F709A7F01922BBFE06F3E5F00975
:10318000F31922C3E49FFFE49EFEE49DFDE49CFC52
:1031900022E0FCA3E0FDA3E0FEA3E0FF22E2FC08A6
:1031A000E2FD08E2FE08E2FF22E493FC740193FDD5
:1031B000740293FE740393FF22E0F8A3E0F9A3E006
:1031C000FAA3E0FB22E2FB08E2F908E2FA08E2CB0C
:1031D000F822E493F8740193F9740293FA74039358
:1031E000FB22ECF208EDF208EEF208EFF222E6FB29
:1031F00008E6FA08E6F922EBF608EAF608E9F6220C
:10320000E0FBA3E0FAA3E0F922F8E0FBA3A3E0F9D6
:1032100025F0F0E582158270021583E0FA38F0227D
:10322000F8E0FBA3A3E025F0F9F0E5821582700237
:103230001583E038FAF022EBF0A3EAF0A3E9F022DC
:10324000E2FB08E2FA08E2F922EBF208EAF208E906
:10325000F222E493FB740193FA740293F922496415
:103260006C65005472616E736D69745F4D65737344
:10327000616765005365745F4C6F676963616C5F7C
:103280004164647265737300436F6E6E65637400AE
:10329000446973636F6E6E656374005374616E642A
:1032A0006279005374616E6462795F416C6C0052A4
:1032B00065636F72645F43757272656E7400526508
:1032C000636F72645F43757272656E745F4F66669A
:1032D000005365745F54696D65725F50726F6772F9
:1032E000616D00436C6561725F54696D65725F501A
:1032F000726F6772616D004765745F4D656E755FD3
:103300004C616E677561676500416E6E6F756E63C7
:10331000655F4D656E755F4C616E677561676500D1
:10332000436F6E74726F6C5F4465636B0053656CC2
:103330006563745F54756E65725F53657276696319
:103340006500436F6E74726F6C5F54756E657200CA
:1033500053656E645F56656E646F725F436F6D6D2B
:10336000616E640042726F6164636173745F56657D
:103370006E646F725F436F6D6D616E640056656E53
:10338000646F725F52656D6F74655F427574746FC0
:103390006E5F507265737365640056656E646F721C
:1033A0005F52656D6F74655F427574746F6E5F52C6
:1033B000656C656173656400526571756573745FF2
:1033C0004D656E7500557365725F436F6E74726FF5
:1033D0006C5F5072657373656400557365725F430B
:1033E0006F6E74726F6C5F52656C656173656400BB
:1033F000526571756573745F53797374656D5F4160
:103400007564696F5F4D6F646500557064617465C4
:103410005F4465766963655F496E666F00526571EA
:10342000756573745F496D6167655F566965775F40
:103430004F6E00526571756573745F546578745F83
:10344000566965775F4F6E00416E6E6F756E63658E
:103450005F4163746976655F536F7572636500538E
:1034600065745F496E6163746976655F536F7572E9
:10347000636500526571756573745F446973706C40
:1034800061795F4F53445F537472696E6700496E90
:10349000666F726D5F4D656E755F537461747573A1
:1034A000005365745F53797374656D5F417564692A
:1034B0006F5F4D6F6465005265706F72745F526527
:1034C000636F72645F537461747573005265706FDB
:1034D00072745F54696D65725F53746174757300C3
:1034E0005265706F72745F54696D65725F436C658D
:1034F000617265645F53746174757300556E7375A2
:1035000070706F727465645F4D6573736167650099
:10351000496D6167655F566965775F4F6E005465F9
:1035200078745F566965775F4F6E004163746976A2
:10353000655F536F7572636500496E616374697688
:10354000655F536F7572636500526571756573745D
:1035500065645F666F725F5374616E64627900497F
:103560006E666F726D65645F4D656E755F4C616E02
:1035700067756167650052656365697665645F5666
:10358000656E646F725F436F6D6D616E640052654E
:103590006365697665645F56656E646F725F5265D8
:1035A0006D6F74655F427574746F6E5F5072657392
:1035B0007365640052656365697665645F56656E20
:1035C000646F725F52656D6F74655F427574746F7E
:1035D0006E5F52656C656173656400446973706CFD
:1035E00061795F4F53445F537472696E6700496E2F
:1035F000666F726D65645F4D656E755F537461745F
:1036000075730052656365697665645F55736572AD
:103610005F436F6E74726F6C5F5072657373656435
:103620000052656365697665645F557365725F43D3
:103630006F6E74726F6C5F52656C65617365640068
:1036400053797374656D5F417564696F5F4D6F6425
:10365000655F536574004465766963655F496E66AE
:103660006F5F4368616E676564005365745F537490
:103670007265616D5F506174680052657175657344
:103680007465645F5265636F72645F4375727265DF
:103690006E74005265717565737465645F5265631D
:1036A0006F72645F43757272656E745F4F66660019
:1036B0005265717565737465645F5365745F5469B1
:1036C0006D65725F50726F6772616D0052657175E2
:1036D00065737465645F5365745F54696D65725F8B
:1036E00050726F6772616D5F5469746C65005265EA
:1036F000717565737465645F436C6561725F54696D
:103700006D65725F50726F6772616D0052657175A1
:1037100065737465645F666F725F4D656E750052A8
:1037200065717565737465645F436F6E74726F6CF9
:103730005F4465636B0053656C65637465645F54D7
:10374000756E65725F536572766963650052657167
:103750007565737465645F436F6E74726F6C5F54EC
:10376000756E6572005265717565737465645F6628
:103770006F725F53797374656D5F417564696F5FD4
:103780004D6F646500526F7574696E675F4F666652
:1037900000443D3078253032582044656570204320
:1037A0006F6C6F722044657465637465640D0A0004
:1037B000443D3078253032582034204F7574707570
:1037C0007420537570706F72740D0A00443D307828
:1037D000253032582054782054524547203D20301F
:1037E00078253032580D0A004572723A204E3D302D
:1037F000782530325820414B535620524459202DC1
:10380000204D4355204949432025640D0A00457247
:10381000723A204E3D30782530325820414B535675
:103820002072656164202D204D4355204949432075
:1038300025640D0A004572723A204E3D30782530DD
:10384000325820414B53562072656164202D204B25
:1038500065792057726F6E670D0A004572723A20C3
:103860004E3D3078253032582054782052692072ED
:10387000656164202D204D4355204949432025642E
:103880000D0A004572723A204E3D3078253032588C
:1038900020424B53562072656164202D20444E20F7
:1038A0004444432025640D0A004572723A204E3D7F
:1038B00030782530325820424B535620726561646F
:1038C000202D204B65792057726F6E670D0A0045D9
:1038D00072723A204E3D307825303258205278208E
:1038E00052692072656164202D20444E2044444377
:1038F0002025640D0A004572723A204E3D3078252D
:10390000303258204B5356204649464F207265614D
:1039100064202D20444E204444432025640D0A0099
:103920004572723A204E3D30782530325820454459
:1039300049442062302072656164202D20444E206D
:103940004444432025640D0A004572723A204E3DDE
:103950003078253032582045444944204368656317
:103960006B206661696C65642C2070454449445B3A
:103970003132365D3D307825303258203E20380DCA
:103980000A004572723A204E3D3078253032582078
:10399000454449442062692072656164202D2044B9
:1039A0004E204444432025640D0A004572723A209B
:1039B0004E3D3078253032582045444944206368D4
:1039C00065636B73756D206572726F720D0A0057B7
:1039D00061726E3A20443D307825303258204E6F67
:1039E00020455043432064657465637465640A0D23
:1039F00000443D3078253032582045504343206400
:103A000065746563746564205665723D25642E2572
:103A1000640A0D005761726E3A204E6F204465763D
:103A200069636520666F756E640D0A005761726E7A
:103A30003A204E6F20417564696F20537973746525
:103A40006D20666F756E640D0A005761726E3A20C4
:103A5000443D307825303258204550434320457648
:103A6000656E74204D697373696E670D0A00457247
:103A7000723A20443D307825303258204550434337
:103A800020436F6D6D616E642054696D652D6F7597
:103A9000740D0A004572723A2049494320666169F3
:103AA0006C6564202562752C204949434164647229
:103AB0003D307825303262582C205265674164646D
:103AC000723D307825303262580D0A00FF325EFFB9
:103AD0003263FF3274FF3288FF3290FF329BFF3235
:103AE000A3FF32AFFF32BEFF32D1FF32E3FF32F726
:103AF000FF3309FF3320FF332DFF3342FF3350FFE5
:103B00003364FF337DFF339AFF33B8FF33C5FF3390
:103B1000DAFF33F0FF340AFF341DFF3433FF34483B
:103B2000FF345FFF3473FF348EFF34A1FF34B7FFDF
:103B300034CCFF34E0FF34FCFF3510FF351EFF3579
:103B40002BFF3539FF3549FF355FFF3576FF358E61
:103B5000FF35B4FF35DBFF35EEFF3603FF3621FFBF
:103B60003640FF3656FF366AFF367AFF3693FF3609
:103B7000B0FF36CCFF36EEFF370CFF371FFF37366E
:103B8000FF374DFF3765FF3785E490FDB0F0A3F0B8
:103B9000A374FFF0A3F0E4A3F0A3F07F0512B8A88C
:103BA000E4F5207DFF7F0512822A7B027DFF7F05E1
:103BB0001269887D1E7F0212822A7B027D1E7F028F
:103BC0001269887D037F0612822A7B027D031241DF
:103BD000DE7D017F0A126988E4FB7D037F0C126998
:103BE00088E4FB7D0F7F01126988E4F5F1FB7D0419
:103BF0001241DE7D087F06126988D2AF75FF387BDF
:103C0000FF7AAF793812B8B4E4FF12AEFE7D017FBF
:103C1000407E0212984A7BFF7A84795312AA1A7B5B
:103C2000FF7A02790612AA1A7BFF7A84796312AAB4
:103C30001A7BFF7AB979287F0312B8D67B007C07FC
:103C40007DD0127CEB7BFF7A84796812AA1A90FEF1
:103C50000174FFF0A37485F0A3743AF07B017AF845
:103C6000790012B14E7D0C7F0B12822A7B017D0CF4
:103C70007F0B1269887D017F0812822A7B027D01F9
:103C80007F08126988129B5E7D017F0812810B7F7D
:103C90000112B8A87B017AF9790DE4FD12854A7A00
:103CA000F9792E7DB41241B67AF9794F7DB9128532
:103CB0004A7AF979707DE01241B67AF979917DE519
:103CC00012854A7AF979B27DEA1241CE7AF979D32E
:103CD0007DEF12854A7AF979F47DD01241CE7AFAD5
:103CE00079157DD512854A7B017AFA79367DDA120B
:103CF000854A7B017AFA79577DDF12854A7FD01297
:103D000001F91289AD7D7012998B1289927D7E1214
:103D1000998B12899B7D7C12998B7AFA79797D60D7
:103D20001241BE7AFA797B7DE012A1DE7AFA797DC2
:103D30007DE21241BE7AFA797F7DE412A1DE7AFA41
:103D400079817DE61241F37AFA79837DE812A1DE6A
:103D50007AFA79857DEA1241F37AFA79877DEC1255
:103D6000A1DE7B017AFA79897DEE12A1DE90FCF268
:103D7000128984A31288F7128968F01289AD128B18
:103D80006F90FCF21288F774F9F074701289007465
:103D9000F9F07491128990128B6F90FCFE1288F7E3
:103DA00074F9F0A374B212890174F9F074D3128912
:103DB0009012935490FCF212896412890174F9F004
:103DC000A374F412890174FAF07415128999128B94
:103DD0006F90FCFE12896412890174FAF0A37436A4
:103DE00012890174FAF0745712899912935490FE53
:103DF000071289847B017AFA797912B802E490FD7E
:103E0000B0F012896F9408503FEF75F002A4247B44
:103E1000F974FA35F0FA7B01C003C002C0017E00DC
:103E20007C007D211228B874702FF974F93EFA9045
:103E3000FE07EBF0A3EAF0A3E9F0D001D002D00333
:103E400012B80212897680BAE4FFFE12B770EFD37F
:103E50009403E4400690FE41F0800AFFFE12B77022
:103E600090FE41EFF090FE417401F07BFF7A84797F
:103E70007E12AA1A74401288E4E4FD7F9412929391
:103E80001288E8FD7F9412929390F90C7401F0FB74
:103E90001288EA7D107F941292931288E27D117F3E
:103EA000941292931288E87D127F94129293128852
:103EB000E27D137F941292931288E87D147F94120E
:103EC000929390F90C74031288E77D207F941292EC
:103ED000937BFF7A84799B12AA1A90F974E054BFFD
:103EE000F090F995E054BFF090F9B6E054BFF0902F
:103EF000F9D7E054BFF090F9F8E054BFF090FA1908
:103F0000E054BFF090FA3AE054BFF090FA5BE0540E
:103F1000BFF02008030241B0C20890FDB07403F066
:103F2000E4A3F012896F940B4003023FDD12891362
:103F3000704490FDB0E0FC12892430E40C12890832
:103F40008002C333D8FC023FBC75F021EC128927F4
:103F500030E51790FA78E075F01484E5F07074128B
:103F600089088002C333D8FC80411289088002C3CB
:103F700033D8FC023FCD90FDB0E0FF75F0211289EF
:103F80001764056007128913640C703890FDB0E067
:103F900012892430E61D90FA78E075F02884E5F067
:103FA00070311289088002C333D8FCFD7F05127975
:103FB000DE80201289088002C333D8FCFD7F051201
:103FC000822A800F1289088002C333D8FCFD7F0546
:103FD00012810B128976A3E004F0023F2390FA7855
:103FE000E004F0C394C84002E4F07B017AF9790D53
:103FF0001241FB90FDB07401F012896F9403500BD5
:1040000012895412528212897680EE90FDB07403A8
:10401000F012896F940B500B128954121B94128961
:104020007680EEE520B4FF051241E68061E490F968
:1040300004F01241E6700A12B0E9E490F901F08050
:10404000491289425408FFF0BF080790F9037443EE
:1040500080311289425404FFF0BF040790F90374C1
:104060004280201289425402FFF0BF020790F903F8
:104070007441800F1289425401FFF0BF010B90F987
:10408000037440F012ACA08005E490F903F0E52041
:10409000B4FF137D027F0612810B1D7F0612822A58
:1040A0001241C60241277D017F0612810B0D7F065A
:1040B00012822A1289AD12B11CEF604390F901E01F
:1040C000FCB443071241C67D028027ECB4420712BC
:1040D00041D67D04801C90F901E0FCB441071241F7
:1040E000D67D08800DECB4400E7D1E7F0212810B40
:1040F0007D107F0212822A90FDB47401F080287D29
:104100001E7F0212810B90FDB5E0D394C85005E0EC
:1041100004F0801390FDB4E0B4010312AD5EE490AE
:10412000FDB5F090FDB4F090FDB2E025E0F0E0FECA
:104130007D047F06129A29EF60047F0180027F00D0
:10414000EE4FFF90FDB2F0BF7F0EE520B4FF047F7D
:104150001D80027F0212764490FDB3E025E0F0E07E
:10416000FE7D087F06129A29EF60047F0180027F9E
:1041700000EE4FFF90FDB3F0BF7F057F0412764441
:1041800030090AC2097F0112B42412764412570082
:10419000200D03023F1290FA8BE0FF04F0EFD3945E
:1041A000325003023F12C20D7F1D127644023F12AD
:1041B000438701023F127B0112854A7B01227B016A
:1041C00012A1DE7B01227D1E7F0212810B227B0168
:1041D00012854A7B01227D1E7F0212810B227F06FF
:1041E000126988E4FB227D0F7F01129A2990F9045D
:1041F000EFF0227B0112A1DE7B012290FED512722C
:10420000A990FED5127201128A97502890FC2F12A5
:1042100072011247981272011273041247AE1272A1
:104220003B24041272311273D31272011272A07401
:104230000112288490FED512720112734F30E621CC
:104240001273DC7D40128F7590FED512723B2404F0
:104250001272311273D31272011272A074011228F9
:104260008490FED512720112281C14604D14607BDC
:1042700014700302432224FE700302435824056095
:104280000302441990FC2F12720112479812720116
:104290001273041247AE12720112727BE4FD128790
:1042A0001F90FED512720112727B7D0112A78D90B4
:1042B000FED5127201740102441690FED5127201ED
:1042C000129592400302441990FED51272011272A7
:1042D000A012B7EF90FED512720112730412B1DA78
:1042E00090FED5127201740202441690FED512722D
:1042F00001129AC4502A90FED51272011272CB9408
:1043000019EE940050030244191272A012730412A1
:10431000A0E112B81590FED5127201740302441682
:10432000802A90FED512720112730412B11CEF6044
:104330001B90FED51272011272CB9432EE94005093
:10434000030244191272A0740502441690FED5129D
:1043500072011272A002441990FED51272011273FA
:104360000412B883EF601490FED512720112730428
:1043700012B901EF90FED56020801290FED5127226
:104380000112730412B901EF90FED5600C12723B5A
:1043900024041272314402800A12723B2404127205
:1043A0003154FD12288490FED51272011273E394E9
:1043B0002CE5F09401500A90001FE475F001122AD8
:1043C0000512730412B11CEF704F90FED5127201EA
:1043D0001273E3942CE5F09401402E1272F530E153
:1043E0001312B1AE90FED512723B240412723154F6
:1043F000FD12288490FED51272017D80128F759077
:10440000FED51272017402800D90FED512723B240B
:104410000412723154FD12288490FED512720112DA
:10442000727B129FDA400302465E90FED512720143
:1044300012727B127329A3E4F0A37413F012ACE0A0
:1044400090FF80E0B41000400302465E904453F8B1
:104450002828730244830244A40244AB0244B202FB
:1044600044BD0244CD0244E102450602451C02451A
:104470003102454102455602456F02458502459588
:104480000245B41272FB0412740D90FF92E0B40F57
:104490000890FC32740FF08005E490FC32F0127347
:1044A000670245111272FB741980171272FB741A9D
:1044B000801090FED51272017D0402465B1272FBE1
:1044C000741C12737F1272017D4002465B1272FBF4
:1044D0007406F0E4A3F090FED51272017D4002460E
:1044E0005B78267CFC1272727E007F031273EB12E3
:1044F000720112727B12730A12B07F90FED5127293
:10450000017D1002465B1272FB7410F0A31412724C
:10451000611273EB1272017D4002465BE490FC2B4A
:10452000F0741212725A1273EB1272017D4002463D
:104530005B1272FB741312737F1272017D4002468C
:104540005BE490FC2BF0741D12725A1273EB127222
:10455000017D4002465B1272FB741EF0A37402F0F0
:10456000E41272BE90FED51272017D4002465B12CB
:1045700072FB7415F074061272601273EB12720102
:104580007D4002465B1272FB741612737F12720139
:104590007D4002465B90FC2B7401F090FC29741F57
:1045A000F0A37402F0E41272BE90FED51272017D87
:1045B0004002465B90FF811272BD90FC32E06405C0
:1045C0007047A3E0702390FED512720112727B90A7
:1045D000FDEF1272DD12A562EF600302465E90FEEF
:1045E000D51272017D8002465B90FED512720112D7
:1045F000727B90FDEF1272DD12A562EF606090FE9B
:10460000D51272017D8002465B90FC33E0702190F0
:10461000FED512720112727B90FD3B1272DD127395
:10462000551247A2703890FED51272017D80802B02
:1046300090FED512720112727B90FD3B1272DD1258
:1046400073551247A2601790FC32E0FF90FC2DE0FA
:10465000B5070B90FED51272017D80129F5290FE1D
:10466000D5127201127361FD600C129F5290FED53B
:1046700012720112740690FED51272011273C030CC
:10468000E328E912722F54F71273D51272011272D5
:104690007BC0037406127283D003E4FD12A42D9034
:1046A000FED51272017D08029F5290FED512720152
:1046B0001273C030E42EE912722F54EF1273D51228
:1046C000720112727B12730A12B07F90FED51272C1
:1046D0000112727BC00390FD45740CF0E4A3F0A3BB
:1046E0000402478D90FED51272011273C030E63C71
:1046F000E912722F54BF12288490FC29E0B4071AE3
:1047000090FED512720112727B90FDFB7401F0A332
:1047100074FCF0A37433F012B0B490FED5127201A1
:1047200012727B1273AC12728C02479290FED512F9
:1047300072011273C030E517E912722F54DF127341
:10474000D512720112727B90FC2DE0FD02A3BD9088
:10475000FED51272011273C030E73CE912722F5479
:104760007F1228841272FB7418F0A37402F090FC7C
:104770003214F0E4A3F090FED512720112727BC0E5
:104780000390FD457418F0A37402F0A31412728C08
:10479000D003E4FD12A42D2212A6DE12B7EF90FE84
:1047A000D522F0128EAC90FC2DEFF0640F2212B1E6
:1047B000DA90FED52290FE1612889D900006122DEA
:1047C0000390FE1912889D12880212281C24F9B445
:1047D00007004003024D159047E575F003A4C5831B
:1047E00025F0C583730247FA0248DA024B13024BE5
:1047F00071024BCA024C0A024C8690FE19128805BF
:104800001288C420E10302489412880212884CC026
:1048100003C002C001128802128817FDD001D00225
:10482000D00312B5721288021288689432EE940096
:104830005003024D1512880EFF12883C1294D5EFDA
:10484000602A1288021288C430E01912884CC00312
:10485000C002C001128802128817FDD001D002D018
:104860000312B5D51288027408024D121288021282
:104870008817FFE4FD12B35D12880212884CC00352
:10488000C002C001128802128817FDD001D002D0E8
:104890000302B6781288021288C430E01912884CDC
:1048A000C003C002C001128802128817FDD001D0D7
:1048B00002D00312B5D512880212884CC003C00280
:1048C000C001128802128817FDD001D002D0031255
:1048D000B5931288027405024D12128802128817CD
:1048E000FFE4FD12B35D128802128817124D219069
:1048F000FE1630E61E12880512884CC003C002C0A6
:1049000001128802128817FDD001D002D00312B51F
:10491000F6801C12880512884CC003C002C0011228
:104920008802128817FDD001D002D00312B617906A
:10493000FA8FE07002A3E060030249B990FE1912F9
:104940008805124D1660221288A6504190FE191259
:104950008805124D166401703490FA90E004F070EE
:10496000E690FA8FE004F080DE1288A6501F90FED9
:10497000191288051288D312B867EF701090FA9058
:10498000E004F070E490FA8FE004F080DC90FE190F
:104990001288051288D390FDD112887812B78790BB
:1049A000FF80E0FF90FA90E02FF090FA8FE0340063
:1049B000F0E0FEA3E0FF12AAA5E490FF88F012AA9F
:1049C000677C017D0012291F90FF88E02480F5821A
:1049D000E434FFF583EDF090FF88E004F0E0C39449
:1049E0000840DB12880212884CC003C002C00112CA
:1049F000880212881790FD75128877D001D002D0F6
:104A00000312B206128802128817FF12883C12B3F2
:104A1000AF12880212884CC003C002C00112880283
:104A200012881790FD7C128877D001D002D0031233
:104A300097A5EF702412880212884CC003C002C0F0
:104A400001128802128817FDD001D002D00312B6DD
:104A5000781288027407024D12128802128817FF1A
:104A600012883C12B3D6128802128817FF12883CB3
:104A70001294D5EF702412880212884CC003C00231
:104A8000C001128802128817FDD001D002D0031293
:104A9000B6781288027407024D1212880212884CEE
:104AA000C003C002C001128802128817FD90FD8366
:104AB000128878D001D002D00312B23212880212CA
:104AC00088D3E94A4B704490FA92E0C39410503472
:104AD000E490FA96F0A3F0128852501812881D1232
:104AE00088CA601090FA97E004F070EB90FA96E0B4
:104AF00004F080E312885240121288841288371220
:104B000088B6800790FA92E04480F0128802740917
:104B1000024D121288021288689407EE9400500326
:104B2000024D1512884CC003C002C0011288021247
:104B30008817FDD001D002D00312B2DFEF90FE162D
:104B4000600B1288051288D9740A024D121288056A
:104B500012884CC003C002C001128802128817FDDF
:104B6000D001D002D00312B6781288027407024D29
:104B70001212880212A498EF70311288021288680B
:104B8000940AEE94005003024D15128843C003C0EE
:104B900002C001128802128817FDD001D002D00392
:104BA00012B6781288027407024D12128802128817
:104BB0000E124D2190FE1630E608128805740D0283
:104BC0004D12128805740B024D1212880212884C85
:104BD000C003C002C001128802128817FDD001D0A4
:104BE00002D00312B5B412880212884CC003C0026E
:104BF000C001128802128817FDD001D002D0031222
:104C0000B593128802740C024D1290FE1912880599
:104C10001288C430E14C128802128868944BEE94DA
:104C2000005003024D151288D912A498EF600302B8
:104C30004D1512880212A498EF6003024D151288D8
:104C40000212884CC003C002C001128802128817E9
:104C5000FDD001D002D00312B658128802740702A8
:104C60004D1212880212884CC003C002C001128883
:104C700002128817FDD001D002D00312B658128854
:104C8000027407024D12128802128817FF12B6B67C
:104C900090FA93EFF030E54F12880212880EFF125F
:104CA000883C12AF7012880290FF80E0FDA3E09074
:104CB000FD66F012006EEF90FE1660081288057413
:104CC0000B024D1212880512884CC003C002C001AD
:104CD000128802128817FDD001D002D00312B678D4
:104CE0001288027407802B12880212886894FAEEE8
:104CF00094004021128843C003C002C00112880200
:104D0000128817FDD001D002D00312B678128802A3
:104D1000740712288422900019122D0312B867EF2D
:104D200022FF12B6B690FA93EFF0220000000000C6
:104D300000000000000000000000000000D6098014
:104D4000A020E02D101060A2000403000000188CC9
:104D50000AD08A20E02D10103E96000403000000C7
:104D6000188C0AD08A20E02D10103E960010090001
:104D7000000018011D007251D01E206E2855001031
:104D8000090000001E011D8018711C1620582C25DA
:104D90000010090000009E8C0AA01451F016002695
:104DA0007C43000403000000988C0AA01451F01604
:104DB00000267C43001009000000988C0AA01451C2
:104DC000F01600267C43000403000000188C0AA0A3
:104DD0001451F01600267C4300100900000018183A
:104DE000154028B2F016004CF84300040300000000
:104DF0009818154028B2F016004CF843001009002E
:104E000000009818154028B2F016004CF843000432
:104E1000030000001818154028B2F016004CF843A3
:104E2000001009000000181815A01451E02D1020E2
:104E30007C96000403000000181815A01451E02D02
:104E400010207C9600100900000018023A801871AA
:104E5000382D40582C450010090000001E8C0AD047
:104E600090204031200C4055000403000000188CB5
:104E70000AD090204031200C40550010090000005D
:104E800018011D00BC52D01E20B828554010090042
:104E900000001E011D80D0721C1620102C258010D1
:104EA000090000009E8C0AA02051201810187E23B3
:104EB000000403000000988C0AA02051201810184C
:104EC0007E23001009000000988C0AA020512018B1
:104ED00010187E23000403000000188C0AA0205143
:104EE000201810187E230010090000001818154023
:104EF00040B220181030FC23000403000000981872
:104F0000154040B220181030FC23001009000000AA
:104F10009818154040B220181030FC2300040300FC
:104F200000001818154040B220181030FC23001063
:104F300009000000181815A0205140312018805594
:104F40000004030000001E1815A020514031201855
:104F500080550010090000001E023A80D072382DE2
:104F600040102C458010090000001E011D803E737A
:104F7000382D407E2C458010090000001E011D8048
:104F8000D072382D40102C458010090000001E0101
:104F90001D80D072382D40102C4580100900000073
:104FA0001E3B2A4028B2E02D1060F8960004030052
:104FB0000000183B2A4028B2E02D1060F89600103F
:104FC0000900000018302A4040B24031203000551E
:104FD00010040300000018302A4040B24031203055
:104FE000005510100900000018201C8080711C550D
:104FF0002020A8750410090000009A023A80D0729F
:105000001C1620102C258010090000009E023A007A
:10501000BC52D01E20B828554010090000001E18B0
:1050200015D090204031200C4055000403000000B2
:10503000181815D090204031200C40550010090060
:105040000000181815D09020201810187E23000496
:1050500003000000981815D09020201810187E2307
:1050600000100900000098023A8018711C162058A0
:105070002C250010090000009E023A007251D01E3B
:10508000206E28550010090000001E1D15D08A2032
:10509000E02D10103E96000403000000181D15D0EE
:1050A0008A20E02D10103E96001009000000181D07
:1050B00015A01451F01600267C43000403000000E4
:1050C000981D15A01451F01600267C43001009000D
:1050D000000098302AD090204031200C4055000428
:1050E0000300000018302AD090204031200C405599
:1050F00000100900000018302AA0205120181018B4
:105100007E2300040300000098302AA020512018BC
:1051100010187E23001009000000983B2AD08A2036
:10512000E02D10103E96000403000000183B2AD02A
:105130008A20E02D10103E96001009000000183B58
:105140002AA01451F01600267C430004030000003E
:10515000983B2AA01451F01600267C430010090049
:1051600000009800FFFFFFFFFFFF0017100109017B
:10517000000000000E0103807341782A7C119E59C3
:10518000479B271050542108000101010101010132
:10519000010101010101010101011D007251D01E37
:1051A000206E28550010090000001E8C0AD08A20AD
:1051B000E02D10103E9600040300000018000000CF
:1051C000FC0045502D48444D492D52580A202000DE
:1051D0000000FD003B3D0F2E08000A20202020206B
:1051E0002001AB02031D714A84051314010203114F
:1051F0001210230907078301000065030C0010004B
:10520000023A801871382D40582C450010090000D2
:10521000001E011D8018711C1620582C2500100935
:105220000000009E011D00BC52D01E20B828554031
:1052300010090000001E011D80D0721C1620102CC9
:10524000258010090000009E8C0AD090204031205B
:105250000C4055000403000000180000000000008E
:1052600000001E8102031112040907070100000358
:105270000C001000881E097F071707503F06C04F1B
:10528000000090FE0A1272A9900006122D0390FEF3
:105290000D1272A990FE0D12723B4A4B700302561A
:1052A000EA90FE0A127201128A97400E90FE0A12CC
:1052B000720112734F70030253E090FE0A127201E2
:1052C000127254C003C002C00190FE0A1272011291
:1052D0007243D001D002D00312B65890FE0A127267
:1052E0003B240412723154FD12738F127201127238
:1052F00054C003C002C00190FE0A12720112724330
:10530000D001D002D00312B59390FE0A127201129E
:105310007254C003C002C00190FE0A1272011272E0
:1053200043D001D002D0031256EB12720112730463
:1053300012B1DA90FE0A1272011272A012734F308B
:10534000E70A90FE0A1272017D80802190FE0A1207
:10535000720112734F30E62390FE0D12723B24014E
:10536000127231444012738F1272017D40128F7598
:1053700090FE0A12720174020253D490FE0A127255
:105380000112734F90FE0A30E545A3A3E07D201281
:105390008F7590FE0A1272011273041256F2127285
:1053A00001127254C003C002C00190FE0A127201C1
:1053B000127243D001D002D0031256F912723B246C
:1053C0000412723112738D12720112733880051239
:1053D0007201740112288490FE0A1272011273DCA9
:1053E00090FE0A12720112281C1470030255A214B6
:1053F00070030255BB1470030255D4147003025697
:105400004A14700302565424056003025685127232
:1054100054C003C002C00190FE0A1272011272430E
:10542000D001D002D0031256EB1272011273041293
:10543000B1DA90FE0D12720112281C70411273F243
:1054400090FE0A30E40C12723B24051272314410B3
:10545000800A12723B240512723154EF1228849094
:10546000FE0D1272011273F290FE0A30E50302552E
:105470004D12723B240512723154DF02555790FED3
:105480000A12723B240512723154EF12288454DF41
:1054900012738F127201127254C003C002C00190C5
:1054A000FE0A127201127243D001D002D0031256CA
:1054B000F91272011273041256F21272011272542E
:1054C000C003C002C00190FE0A127201127243D0E2
:1054D00001D002D00312AC18EF701090FE0A1272C5
:1054E0003B2405127231441002555790FE0A127285
:1054F00001127254C003C002C00190FE0A12720170
:1055000012724390FD7C12732CD001D002D0031292
:1055100097A5EF700F90FE0A12723B2405127231AC
:105520004410803390FE0A12723B240512723154EB
:10553000EF12288490FE0A127201127419FF7B0187
:105540007AFF79801294D5EF701090FE0A12723BA8
:105550002405127231442002288490FE0A12723B04
:10556000240512723154DF12288490FE0A1272014F
:10557000127254C003C002C00190FE0A12720112DE
:105580007243D001D002D00312B63890FE0A1272D4
:105590000112730412B1DA90FE0A12720174010250
:1055A000568090FE0A127201129592400302568EA6
:1055B00090FE0A127201740202568090FE0A127264
:1055C00001129AC4400302568E90FE0A12720174B0
:1055D0000302568090FE0D12720112281CD3940310
:1055E000500302568E90FE0A127201127254C003CA
:1055F000C002C00190FE0A127201127243D001D0A3
:1056000002D00312B5D590FE0A1272011273041271
:10561000A0E190FE0A127201127254C003C002C0CF
:105620000190FE0A127201127243D001D002D0031F
:1056300012B55190FE0A12723B24041272314401D9
:1056400012738F1272017404803690FE0A12720176
:105650007405802C90FE0D1272011272F590FE0AF4
:1056600030E11312723B240412723112738D1272E4
:1056700001127338800A12723B240412723154FDF5
:10568000122884800990FE0A1272011247B590FE1A
:105690000A12720112A06090FE0A12723B50092495
:1056A0000412723144108007240412723154EF1234
:1056B000288490FE0A127201127361FD600C129F21
:1056C0005290FE0A12720112740690FE0A127201C2
:1056D0001273C0FF601490FE0D1272284F12738F68
:1056E000127201900003E41228962212B63890FE3E
:1056F0000A2212A0E190FE0A2212B55190FE0A225F
:1057000012B3FD90FF05EFF0F47003025A22E0FFA0
:1057100090FC95E0FE04F074812EF582E434FCF5F3
:1057200083EFF090FC95E0D39412400E7BFF7A6CEF
:10573000798E12AA1AE490FC95F090FF05E0FF64C0
:105740000A6008EF640D6003025A22E490FC95F0B1
:1057500090FBFA74FFF0A3746CF074AA127C2574A9
:10576000FFF07480127C2574FCF0A37479127C26FF
:1057700074FCF0A3747B127C2674FCF0A3747D127D
:105780007C2674FCF0A3747FF0127BBA1266EFE4FF
:1057900090FC84F07A6C79B9127B85701E7A6C79F2
:1057A000BD125A28127CC6FD90FC7EE0FB12B0149C
:1057B00090FC7AE090FC93F0025A227A6C79E51220
:1057C0007B85703B7A6C79E9127C2D12AA1AD23251
:1057D00090FC7AE090FE6CF090FE6DE0FBA3E0FAA6
:1057E000A3E0F9EA494B7003025A2290FE6DA3A38D
:1057F000E0F5828A837D10E4FF122DB6025A227AE8
:105800006D7903127B92701E7A6D7907125A289077
:10581000FC7EE090FC81F0127CC690FDA7127B78A4
:10582000129DAB025A227A6D7938127B9260030284
:1058300058BE7A6D793C127C2D90FC7B127C7C905A
:10584000FC7DE0FFA3E090FBD0CFF0A3EFF012AA25
:105850001AD390FC7EE0941290FC7DE09400400608
:10586000127BDB12AA1A90FC7AE04401FFC00712F7
:105870007BB5A3E0FFA3E090FDA7CFF0A3EFF0D0AE
:1058800007129DABEF6003025A2290FC96F0A3F042
:1058900090FC7D127C3F5023ED540F7006127CD09B
:1058A00012AA1A90FC97E054077003125B5A125B1D
:1058B0002B70DD90FC96E004F080D50259BF7A6D24
:1058C00079A8127B9F70247A6D79AC125ADE129DF2
:1058D000ABEF6003025A22127CD7FEEF6E127BAC54
:1058E000125B4D6003025A220259ED7A6D79EC1277
:1058F0007B9F70257A6D79F0125ADE129DABEF60B6
:1059000003025A22127CD7F4FEEF5E127BAC125BCC
:105910004D6003025A220259ED7A6E7927127BC13B
:105920007017127BCE7A6E792B125A5B90FC80E056
:10593000127B67129D1B025A227A6E795C127BC120
:1059400060030259C5127BCE7A6E7960125A5BD31E
:1059500090FC80E0941290FC7FE094004006127B63
:10596000DB12AA1A90FC7AE04401FFC00790FC7D8C
:10597000E0FCA3127BB8A3E0FFA3E090FD60CFF0B2
:10598000A3EFF0D007129D1BEF6003025A2290FC98
:1059900096F0A3F090FC7F127C3F5023ED540F70E3
:1059A00006127CD012AA1A90FC97E05407700312DA
:1059B0005B5A125B2B70DD90FC96E004F080D512F0
:1059C0007CD0025A1F7A6E7997127C897025127BDF
:1059D000CE7A6E799B125A8E129D1BEF7044127C08
:1059E000E1FEEF6E127B67129D1BEF7035127C514A
:1059F000025A1F7A6E79D2127C897026127BCE7A77
:105A00006E79D6125A8E129D1BEF7016127CE1F43D
:105A1000FEEF5E127B67129D1BEF7006127C511227
:105A2000AA1A90FF05E0FF227BFF90FC79E0FFA31C
:105A3000E090FBCCCFF0A3EFF090FC7BE0FFA3E085
:105A400090FBCECFF0A3EFF090FC7DE0FFA3E090C1
:105A5000FBD0CFF0A3EFF012AA1A227BFF90FC79C3
:105A6000E0FFA3E090FBCCCFF0A3EFF090FC7DE053
:105A7000FFA3E090FBCECFF0A3EFF090FC7FE0FF20
:105A8000A3E090FBD0CFF0A3EFF012AA1A227BFF85
:105A900090FC79E0FFA3E090FBCCCFF0A3EFF09077
:105AA000FC7DE0FFA3E090FBCECFF0A3EFF090FCF5
:105AB0007FE0FFA3E090FBD0CFF0A3EFF012AA1A93
:105AC00090FC7AE04401FF90FC7DE0FCA3E0FD7BCC
:105AD000017AFC798190FD60E4F0A304F0227BFF61
:105AE00090FC79E0FFA3E090FBCCCFF0A3EFF09027
:105AF000FC7BE0FFA3E090FBCECFF0A3EFF090FCA7
:105B00007DE0FFA3E090FBD0CFF0A3EFF012AA1A44
:105B100090FC7AE04401FF90FC7CE0FD7B017AFC84
:105B2000798190FDA7E4F0A304F0227BFF7A6D79E0
:105B30009E90FC97E02481F582E434FCF583E090AC
:105B4000FBCCF012AA1A90FC97E004F02290FDA77B
:105B5000E4F0A304F0129DABEF227BFF7A6D799CF9
:105B600012AA1A225FFFE0FBA3E0FAA3E0F990007B
:105B700001EF12289690FCA3E02402FFE433FE908C
:105B8000FC9AE0FBA3E0FAA3E0F98F828E8312284F
:105B900035FF90FCA2E02402FDE433FC90FC9DE084
:105BA000FBA3E0FAA3E0F9228D828C83122835FF53
:105BB00090FC9AE0FBA3E0FAA3E02480F9E43AFA2F
:105BC00090FCA3E02290FCA3E0FFF5827583000225
:105BD00028358F828E83122835FF22E429F9EA3492
:105BE00001FA12281C54FE12288490FC9AE0FBA3B0
:105BF000E0FAA3E022E0FE04F08E82758300EF124B
:105C0000289690FCA17401F022FDEE33FC8D828C6D
:105C10008302283590FCA2E0FF7E0090FE42E0FC6B
:105C2000A3E0FD2290FCA2E0FF90FE43E02FFF9056
:105C3000FE42E0340022FE04F0EE7C0029F9EC3A4A
:105C4000FAEF02288490FD207401F0A374FCF0A305
:105C500074A8F090FCB1E0F9A3E0FAA3E090FD2372
:105C6000C9F0A3EAF0A3E9F02290FCA5541FFEEFCF
:105C70002EF02290FCA7E0FE04F08E82758300EFE8
:105C800002289690FE42E0FEA3E0FF22FF90FE4035
:105C9000E02FF090FE43E004F022122896E490FEFC
:105CA00040F090FE42F0A3F022541FFEEF2E90FC35
:105CB000A4F090FCA2E004F02290FCA5E0FF90FC90
:105CC000A3E0FED39F2290FE42E004F022F090FD7C
:105CD000B97401F0A374FCF0A374A7F090FCAB229C
:105CE000E0FFC390FE43E09F7480F890FE42E064C2
:105CF00080982290FCA3E004F022C39F7480F8EC0B
:105D000064809822E429F9EA3401FA12281C54FD2F
:105D100002288490FCA3E0FF04F08F8222FF04F0AD
:105D20007E00E92FF9EE3AFA2290007E12283564BF
:105D30000122900001EF12289690FC9A22F8AC0202
:105D4000AD037BFF228D828C83EF022896C3ED9FEB
:105D5000EE6480F8EC6480982290FCA37484F022B6
:105D600012288490FCA3E02401FFE433FE90FC9A07
:105D700022EF900002022896900001122835FF9031
:105D8000FC9A2290FCA4E0FF90FCA2E02290FCA8E8
:105D9000E02402FDE433FC90FCAE2290FCA2E0FD86
:105DA0007C00EF2D22EF2402FFE43EFE2212281C8D
:105DB000FF90FCA2E02401222480F9E43AA801FC2F
:105DC000AD032290FCA27484F02290FE40E014F413
:105DD000FF90FC9A2290FCA2E02402FFE433FE2212
:105DE0002FF582E43EF583022835EF2405FDEE33DE
:105DF000FCE92DF9EA3CFA02281C90FCA3E0FD9096
:105E0000FE43E02DFD229001000228357E007F80B8
:105E10000227F690FE41E064032290002302283519
:105E2000EF12288490FC9A229000240228359000DA
:105E3000250228359000011228356D2290000212AB
:105E400028356F228F828E830228352FFFEE3CFE8D
:105E5000E0FBD3EF9B7480F86E9822C4135407FDC7
:105E6000EF541F2D2290FCB4A3A3E02405F9E43ADB
:105E7000FA02281C7E00FDEE33FC90FC9A221228C8
:105E800084448012288490FCB422122884EF2406D3
:105E9000FFEE33FE90FC9A22C3947FEE64809480E0
:105EA00022900082022835A3F0A3EBF0A3222480E5
:105EB000F9E43AFA22900036022835900037022899
:105EC00035FC8D82F5830228359000060228359036
:105ED000FCA7E0C3941E2290FCA8E0C3942D22905E
:105EE000FCA9E0C394052290FCA2E02403F02290D8
:105EF000FCA5E0FF90FCA3E0D39F2290FCA9E0C3A7
:105F0000941F22740512288490FCB7222400F9EA19
:105F10003401FA02281C2DF582E43CF58302283571
:105F200090FCA2E0240DFFE433FE22541FFF90FEFC
:105F300043E02FF02290007E0228351231387E0097
:105F40007F037D0022900083022835E0FFFDC3908F
:105F5000FE43E09D22541FFEEF2E90FCA4F0229001
:105F6000FE42E0FCA3E0F5822290FCA8E0F58275F9
:105F700083002212288490FCB12290FD12EBF0A342
:105F8000EAF0A3E9F0122BE390FBB5122CC69000C7
:105F900004122C0390FBB9122CC6900008122C039B
:105FA00090FBBD122CC690000C122C0390FBC1126A
:105FB0002CC6900010122C0390FBC5122CC6E49046
:105FC000FD18F090FD18E0FFD3944F400302626685
:105FD000EFC39410500302606290FD15128D4AF9D0
:105FE000A3E02408128D62122C03C00790FD15A3B4
:105FF000A3A3E0240D128D62122C8AD007EB128D20
:106000007BC00790FD15128D4AF9A3E02402128D82
:1060100062122C8AD007128DA5C00790FD15128D33
:106020004A128D5F122C8AD007128DA590FD19128D
:106030008D2F7801122BD0C004C005C006C00712F6
:106040008D32781F122BA9D003D002D001D00012BC
:106050008D6EC00790FD15128D4A128D5FD007120C
:106060002C4D90FD15128D4A128D5F122C03128D4E
:10607000B290FD19128D24FBC000C001C002C00304
:1060800090FBB5128D357805122BD0C004C005C029
:1060900006C00790FBB5128D35781B122BA9D003D3
:1060A000D002D001D000128D6ED003D002D001D02A
:1060B00000128D52128DB290FD18E0D39413504807
:1060C000A3128D24FBC000C001C002C00390FBB925
:1060D000128D35122B9C90FBC1128D24128D87C01E
:1060E00004C005C006AB07128D13128D87D002D0F5
:1060F00001D000128D6EEF2499FFEE3479FEED345D
:1061000082FDEC345A0261E490FD18E0D3942750EC
:106110002EA3128D24FBC000C001C002C003128D4B
:1061200013128D7B90FBC1128D24128D7BEF24A165
:10613000FFEE34EBFEED34D9FDEC346E0261E490F9
:10614000FD18E0D3943B506FA3128D24FBC000C018
:1061500001C002C00390FBC1128D16128D87C004CE
:10616000C005C006AB07A3128D3590FBB9A3A3A34E
:10617000E0128D87D002D001D000128D6EC004C015
:1061800005C006AB0790FBC1128D3590FBBD128D8B
:1061900024128D87D002D001D000EB4FFFEA4EFED3
:1061A000E94DFDE84CFCEF24DCFFEE34BCFEED34A1
:1061B0001BFDEC348F802D90FD19128D24FBC00047
:1061C000C001C002C003128D13128D7B90FBC1125F
:1061D0008D24128D7BEF24D6FFEE34C1FEED3462A8
:1061E000FDEC34CAFCD003D002D001D000128D5295
:1061F000128DB2128D3290FBC5128D24FBEF2BFF56
:10620000EE3AFEED39FDEC38FC128DB290FBC11276
:106210008D35A3122CC690FBBD128D35A3122CC652
:1062200090FBB9128D35781E122BD0C004C005C06A
:1062300006C00790FBB9128D357802122BA9D00346
:10624000D002D001D000128D6EA3122CC690FBB5E7
:10625000128D35A3128D2F90FBB5122CC690FD1810
:10626000E004F0025FC390FD12128D4AF9C002C033
:1062700001122BE390FBB5128D24128D53D001D067
:1062800002128DB8128D4A2404F9E43AFAC002C011
:1062900001122BE3128D21128D53D001D002128DE9
:1062A000B8128D4A2408F9E43AFAC002C001122B50
:1062B000E390FBBD128D24128D53D001D002128DBC
:1062C000B8128D4A240CF9E43AFAC002C001122B2C
:1062D000E390FBC1128D24128D53D001D002128D98
:1062E000B8128D4A2410F9E43AFAC002C001122B08
:1062F000E390FBC5128D24128D53D001D002022CE5
:1063000033E50D2454F582E434FCF583E0050D22D9
:1063100090FC5130270390FC54E475F001123209CF
:1063200002281C2020E97F2ED2208018EF540F2451
:1063300090D43440D4FF30240BEF24BFB41A005063
:10634000032461FFE50E6002150E0511E5117002D0
:10635000051030270E90FC51E475F001123209EF60
:1063600002288402B44B7403D2278003E4C227F5C9
:106370000D90FC51123237E4F50EF510F511E50ED3
:1063800060077F2012634480F5750FFFC221C22091
:10639000C222C223C225C226C228126310FF700D7A
:1063A0003027057F00126355AF11AE1022B4255F70
:1063B000C2D5C224126310FF24D0B40A00501A754B
:1063C000F00A780E30D50508B6FF0106C6A426F6F9
:1063D00020D5047002D22380D924CFB41A00EF5004
:1063E00004C2E5D224026556D22180C6D22080C0E4
:1063F000D22280BCD2D580BAD22580B47F2012634D
:10640000442022077401B50E0040F1126301FF120F
:10641000634402637ED228D2268095126301FB1268
:106420006301FA126301F94A4B700679277A667B99
:10643000FF20222EE50E602A7E008E8275830012D8
:10644000283560060EEE650F70F0C2D5EBC0E0EAAD
:10645000C0E0E9C0E0EE12659DD0E0F9D0E0FAD0EE
:10646000E0FB12281CFF60AAEBC0E0EAC0E0E9C034
:10647000E0126344D0E02401F9D0E03400FAD0E027
:10648000FBE50F0460DCD50FD980877BFF7A657947
:1064900099D222809C791080027908C226C2288075
:1064A00008D2D5790A8004790AC2D5E50F047002B2
:1064B000F50FE4FAFDFEFF126301FC7B08202113B7
:1064C000126301FD7B1030200A126301FE1263018A
:1064D000FF7B20EC3382D592D55013C3E4302006E5
:1064E0009FFFE49EFEE42021039DFDE49CFCE4CBA1
:1064F000F8C221EC700CCFCECDCCE824F8F870F3C4
:106500008017C3EF33FFEE33FEED33FDEC33FCEBCE
:1065100033FB994002FB0FD8E9EB302105F8D0E0BE
:10652000C448B221C0E00AEC4D4E4F78207B007089
:10653000C2EAB50F0040BCC0E012659FD0F0D0E0C9
:10654000202104C4C0E0C4B221C0F012632DD0F0F9
:10655000D5F0EB02637E122D8C641B536495586357
:10656000EC4C63E84264994F64A14464A14964011E
:106570004364A755648B46648B45648B47664750DC
:1065800063F02D63F42E64172B63F82364152066E3
:10659000302A63B0480000640F3F3F3F00790AA2F1
:1065A000D5202314302509B910020404B9080104C8
:1065B000A2D52026025001042022689222B50E00A6
:1065C0005034C0E07F203023197F30A2227226721F
:1065D00025500F1265F6C222C226C225C2287F307E
:1065E000800F302503E9C0E0126344302503D0E07A
:1065F000F9D0E0B50ECC3025177F30B9100C1263FE
:10660000447F583024077F788003B908031263441D
:106610003022057F2D0263447F202028F87F2B2025
:1066200026F322922280CF286E756C6C2900D2212D
:106630001263013021F8C221780E30D50108F6022C
:1066400063B02D504349581263012403B405004040
:1066500001E490664293126335743A126335D22393
:10666000750E04026495E508302C0104F8232824F3
:10667000FAF582E434FBF5832290FBF7302C03908B
:10668000FBFAE475F00112320902281C60EAC50C1D
:106690007002150B14C50C202C04FF02B91A90FBD4
:1066A000F774FFF5F0023220FF02B7DBE509600660
:1066B000D509037F0022202C0F12B7C7EF60080511
:1066C0000CE50C7002050B2290FBF7123200122829
:1066D0001CFF60E890FBF7E475F00112320980DCE2
:1066E0001266B6EFC0E01266A8D0E040F3809DD2FB
:1066F0002C8002C22C90FBF7123237E4F50AF50821
:10670000F50BF50C750900C22BC229C22AC22D1245
:106710006679FF7005AF0A7E0022B42530126679D3
:10672000FF24D0B40A00500C75F00AC509A425094D
:10673000F50980E924CFB41A00EF5002C2E50269DE
:1067400054D22A80D8D22980D4D22D80D0EF12669C
:10675000A850081266E0EF600E80A9EFC0E0126654
:10676000B6D0E06F609EEF607412668C80A71266F0
:10677000B6EF6069E5097007050980031266B6EF98
:106780006014202D0E126666E475F001123209EFD6
:10679000122884D509E6202D040508050A80BA12BE
:1067A00066ACEFC0E01266A8D0E0500412668CE43C
:1067B000FF202D0E126666E475F001123209EF1209
:1067C0002884EF70DA202D040508050A808BE5097E
:1067D000600205091266E01266ACEF70C6302C0448
:1067E000E412668CE50A60030267157EFF7FFF22D4
:1067F000202D1174FFFCFDFEFF126666123200129E
:106800002C330508026704D0E080D27900800A7931
:1068100010800679088002790AD22EE50960020507
:1068200009E9C0E01266E0EF60DD1266B6BF2D0434
:10683000D22B8003BF2B091266E0EF60CA1266AC50
:10684000D0E0B40A028033B40802802EBF30277033
:10685000027408C22EC0E01266ACD0E0BF7802809D
:1068600003BF58160509D509028007D50904D22EA1
:10687000800B741080197002740ABF000AEFF8E4EC
:10688000FCFDFEFF026907C0E0EF12668CD0E0F964
:10689000E4FCFDFEFFE9C0E0ECC0E0EDC0E0EEC0CE
:1068A000E0EFC0E01266ACEFF8D0E0FFD0E0FED041
:1068B000E0FDD0E0FCD0F0E8604DB461004007B4EA
:1068C0007B005002C2E524D0503DFA24F650072444
:1068D000F95034240AFAEAB5F000502BCFA9F0A4FD
:1068E0002FFF92D5E9C5F0CEA4A2D53EFE92D5E900
:1068F000C5F0CDA4A2D53DFD92D5E9C5F0CCA4A2AA
:10690000D53CFCC22E808EE8C0E0202D2A202E0827
:10691000050A302B03123183126666123200050815
:1069200020290B202A0DEE8FF01231648009122CE1
:10693000338004EF122884D0E012668C02670420B2
:106940002D101266661232000508E50B850CF01258
:10695000316480E8122D8C67CE53680F5867454C20
:10696000674142671D4868134F681744676E436864
:106970000B4968175567F04667F04567F047674968
:106980002A693F4E0000674D90FEEBEDF0A3EBF05F
:1069900090FEEAEFF014604914607A147003026A02
:1069A0003B147003026A5224FA7003026A86147060
:1069B00003026AC5240B6003026B2A90FEECE0FF21
:1069C000700790FEEBE042FC22EF90FEEBB4020574
:1069D000E042C88004E0F452C890FEEBE0F452FCC0
:1069E0002290FEECE0FF700790FEEBE042FD22EF0C
:1069F00090FCCFB40213128C46FEEF4EFF90FCCFFA
:106A0000F090FCD4E05F42FD22128C4690FCCF1245
:106A10008CF752FD2290FEECE0FF700790FEEBE059
:106A200042FE22EF90FEEBB40205E042D88004E083
:106A3000F452D890FEEBE0F452FE2290FEECE070AF
:106A40000D90FCD6128C46FEEF4E90FCD6F0128CC8
:106A5000FE2290FEECE0FF700790FEEBE042F32296
:106A6000EF90FCD0B40213128C46FEEF4EFF90FC68
:106A7000D0F090FCD7E05F42F322128C4690FCD01D
:106A8000128CF752F322128C95700C90FCDD128C54
:106A90006E90FCDDF08027EC90FCE0B40211128CCB
:106AA0004690FCE0128C8390FCDD128CA0800F12CB
:106AB0008C4690FCE0128C8C90FCDDE05EF090FC4B
:106AC000DDE0F58A2290FEEBE0541CF0A3E0FC70C0
:106AD0001790FCDEE0FE90FEEBE033333354F8FD1C
:106AE000EE4D90FCDEF0803BEC90FCE1B4021E1217
:106AF0008C46128CDAEF4EFF90FCE1F090FCDEE069
:106B0000FE33333354F85FFFEE4FF08016128C469D
:106B100033333354F8F4FEEF5E90FCE1F090FCDE8A
:106B2000E05EF090FCDEE0F5C122128CAB706F905D
:106B3000FEEA128CBE500724FE602C026C8D12B44B
:106B4000E490FEECE0FF700790FEEBE0429B22EF4A
:106B500090FEEBB40205E0429C8004E0F4529C906D
:106B6000FEEBE0F4529B2290FEECE0FF700790FEFB
:106B7000EBE0429722EF90FCD2B40213128C46FE57
:106B8000EF4EFF90FCD2F090FCDFE05F42972212C4
:106B90008C46F4FEEF5E90FCD2F0EE52972290FE0F
:106BA000EAE024FA603A14604914605D24FC700342
:106BB000026C5224076003026C8D90FEECE0FF70C3
:106BC0000790FEEBE0429B22EF90FEEBB40205E063
:106BD000429C8004E0F4529C90FEEBE0F4529B2235
:106BE00090FEECE090FEEB7004E0429422E0F45260
:106BF000942290FEECE0700D90FCDA128C46FEEFD1
:106C00004E90FCDAF0128D0522128C95700C90FCDF
:106C1000DB128C6E90FCDBF08031EC90FCCEB40289
:106C200016128C46C454F0FEEF4EFF90FCCEF0904E
:106C3000FCDB128CA08014128C46C454F0F4FEEFDE
:106C40005E90FCCEF090FCDBE05EF090FCDBE0F5CB
:106C5000AD22128C95700C90FCDF128C6E90FCDFD4
:106C6000F08027EC90FCD2B40211128C4690FCD23A
:106C7000128C8390FCDF128CA0800F128C4690FC4B
:106C8000D2128C8C90FCDFE05EF0128D0C220A4454
:106C90004247434D4420537472696E6720427566C3
:106CA0006665722046756C6C0A0025732025582095
:106CB000255820255820255800627573000A444243
:106CC00047434D44206275733A204275733D255801
:106CD0002C20506F72743D25582C205370656564CC
:106CE0003D25580A00636972000A444247434D44F7
:106CF000206369723A20436F64653D3078253032F5
:106D0000580A00777231000A444247434D442077C5
:106D100072313A2049443D3078253032582C205287
:106D200065673D3078253032582C20446174613DD0
:106D30003078253032580A00726431000A444247E4
:106D4000434D44207264313A2049443D3078253027
:106D500032582C205265673D3078253032582C202F
:106D600053697A653D3078253032582C204461745F
:106D7000613D002852656164206E756D6265722008
:106D80006578636565642061206D6178206F662099
:106D9000256420627974657329000A002000307828
:106DA00025303262582C2000746231000A44424778
:106DB000434D44207462313A2049443D30782530B7
:106DC00032582C205265673D3078253032582C20BF
:106DD0004D61736B3D3078253032582C20446174FE
:106DE000613D00307825303262580A00636231001C
:106DF0000A444247434D44206362313A2049443DAE
:106E00003078253032582C205265673D3078253057
:106E100032582C204D61736B3D3078253032582C20
:106E200020446174613D00777232000A4442474356
:106E30004D44207772323A2049443D307825303233
:106E4000582C205265673D3078253034582C20442A
:106E50006174613D3078253032580A007264320026
:106E60000A444247434D44207264323A2049443D2B
:106E70003078253032582C205265673D30782530E7
:106E800034582C2053697A653D3078253032582C9F
:106E900020446174613D00746232000A44424743F9
:106EA0004D44207462323A2049443D3078253032D6
:106EB000582C205265673D3078253034582C204DB1
:106EC00061736B3D3078253032582C2044617461F9
:106ED0003D00636232000A444247434D44206362EE
:106EE000323A2049443D3078253032582C205265C2
:106EF000673D3078253034582C204D61736B3D3020
:106F000078253032582C20446174613D004552523E
:106F10004F523A20494943206661696C65642025D7
:106F200062752C20494943416464723D30782530B4
:106F30003262582C20526567416464723D30782576
:106F4000303262580A0090FD2FE0FBA3E0FAA3E084
:106F5000F912281CFF90FD32E0FBA3E0FAA3E02227
:106F6000F090FD0BE475F00112296BFE748025F0A2
:106F7000F58274FF3EF5837469F090FD0BE475F0C3
:106F80000112296BFE748025F0F58274FF3EF583B3
:106F900022F912281C04FF90FDA07B00E47A0079FE
:106FA00022F0A304F022F0A3EDF0A3EBF0A3EAF0AB
:106FB000A3E9F02212281C04FF90FD587B00E47A1C
:106FC000007922F0A32290FCE7E47B017AFF79802C
:106FD000F0A322F912281C90FBCCFFE4F0A3EFF001
:106FE00022F9900001022835F912281C7AFF7980D5
:106FF000FF7B0190FD58E4F0A3227B007A00792208
:1070000090FCE7E4F0A322F912281CFF90FE2AE48A
:10701000F0A30422F912281CFFE490FE2AF0A32218
:10702000F990FD0BE0FEA3E0F5828E83022835F98E
:10703000900002122835FF900003122835FD2279B6
:1070400061E7C4F8540FC868FF19E7C454F048FE5C
:10705000E42FFDEE22F9A3E0FFA3E090FCE7CFF0E0
:10706000A3EFF0222FF9EA3EFA900004122835FF30
:10707000900005122835FD2290FD09EFF0E0FE2278
:1070800004F0A3F07D74FF22F990FDA0E4F0A322A8
:1070900012281CFF7B017AFF798090FD0BE0FDA395
:1070A000E090FD58CDF0A3EDF0222401F9E43AFA86
:1070B00002281C7405F0E4A3F07D757F0122E490A2
:1070C000FD0BF0A3F02290FD09E0FFE490FBCEF071
:1070D000A3EFF022F912281C04FF2290FD94E0FD9A
:1070E00090FBCCE4F0A3EDF0A322A3E4F0A3E5220F
:1070F000F07BFF7A3779CC2290FD0BE4F0740AA381
:10710000F0E4A3F0A3F02290FD0CE004F02290FD47
:107110000BE004F02290FDDFE014FF90FDDEE022A2
:1071200090FD0BE0FEA3E0FFC39406EE6480948024
:1071300022D390FD0CE0940090FD0BE0648022903F
:10714000FD0EE004F02290FD0DE004F02204F0A317
:107150007403F07D607F01227480F0E4A3F07DA1D0
:107160007F0122C390FD0EE0940390FD0DE064804A
:1071700094802290FD09E0FF90FBCE2290FF80F0EA
:107180007B017AFF798022C390FE63E094E890FE51
:1071900062E0940322E025E0FF90FD0BE033FE90D7
:1071A000FD0F22A3E024FDF090FD0BE034FFF02260
:1071B000F0A304F07D60FF2290FE29E0FF7401A897
:1071C0000708227BFF7A3A799490FBCCF022E522E3
:1071D00025E0F52222F0A37402F07D747F012224C1
:1071E00007F9E43AFA2290FE10E0FBA3E0FAA3E0EC
:1071F0002404F9E43AFA12281C54FB12288490FE65
:1072000010E0FBA3E0FAA3E0F92290FC32EFF0904B
:10721000FC2AE0FF7E0078337CFC7D017B017AFF55
:1072200079821227F690FE13E0FBA3E0FAA3E02494
:1072300003F9E43AFA02281C90FE10E0FBA3E0FAFE
:10724000A3E022900015122835FD2290001FE4F5DE
:10725000F0122A52900016022D0390FC29F0740FB0
:10726000A3F0E490FC32F090FC2AE0FF7E0078333B
:107270007CFC7D017B017AFF79822290001C022D2B
:1072800003740B90FD45F0E4A3F0A304F0A374FC99
:10729000F0A37432F022900009122D03EA494B2228
:1072A00090001FE4F5F0022A52EBF0A3EAF0A3E904
:1072B000F02290FC29F0A37402F090FC2DE090FCE9
:1072C00032F090FF82E090FC33F02290001FE475D2
:1072D000F0011229B9FEC3E5F02290FD327401F0ED
:1072E000A374FCF0A37434F022900009122D030261
:1072F000281C122D03900004022835E490FC2BF08A
:1073000090FC2922900019022D0390FDE97401F0F0
:10731000A374FCF0A37426F02290FC29F07401A35E
:10732000F090FC2DE090FC322290FD4D7401F0A312
:1073300074FFF0A37480F02290001FE475F0321205
:107340002A527407221228967B007A007900229034
:107350000001022835A37401F0A374FCF0A3744368
:107360002290000202283590FF82E0FF90FC33F06B
:107370007E0078347CFC7D017B017AFF798322F0EA
:10738000A37401F0E490FC32F090FED52244021286
:10739000288490FE0A2290FCA0F090FC9D7401F0DD
:1073A000A374FAF0A37498F090FC2F2290FC29E0CB
:1073B00090FD45F090FC2AE090FD46F0A374012278
:1073C00090000302283590FC29F07401A3F090FF8F
:1073D00092E02254FD12288490FED522900001E410
:1073E00002289690001F122981C3221227F690FED0
:1073F000D522900005022835122D03E9240122121E
:107400002D03E9240222900002E4022896F090FF66
:1074100082E0240390FC2AF0229000150228357B9C
:10742000017AFA79982290FD95126FAB90FD94EF56
:10743000F012A88AE490FF80F090FCE7126FCA1265
:1074400071B0127833126FC612714D127833E41294
:10745000717C90FCE7F0A3127639127078C0069028
:10746000FD95126F58F9127000127158127833D0CE
:10747000E04F90FD09F060137BFF7A39792090FD91
:1074800094E0126FD712717302755B90FD95126FC5
:1074900058F990007E122835FFD3940840141270DA
:1074A000DBE4F0A3EFF07BFF7A39794912AA1A7F67
:1074B000052290FD95126F58F990007E12283590A4
:1074C000FD99F0E4A3F090FD9804F090FD99E0FFA1
:1074D00090FD98E0FED39F4003027572EEC3131235
:1074E000717CE490FCE7F0A31271B0127833126F54
:1074F000C612714D12783390FD98E05401C43333B5
:1075000033548090FF80F0126FC612763912707873
:10751000C006126FC6127158127833D0E04F90FD3A
:1075200009F090FF80E0B4022290FD9AE0701C0404
:10753000F090FD95126F582480F9E43AA801FCAD53
:10754000031271807E007F801227F690FD09E0FF14
:1075500060177BFF7A3979821270DBE4F0A3EFF0D9
:1075600012AA1A90FD09E0FF2290FD98E004F002B3
:1075700074CB90FD95126F58F9E412288490FD9514
:10758000126F58F990000174FF122896900002744F
:10759000FF12289690000374FF122896900004743E
:1075A000FF12289690000574FF122896900006742A
:1075B000FF122896900007E4122896E490FD0AF046
:1075C000A3F0A3F090FD9AE060067E017F008004A6
:1075D0007E007F80C390FD0CE09FEE6480F8127106
:1075E0003898501A90FD95126F58127020FF90FD38
:1075F0000AE02FF012710770CB12710E80C690FD59
:107600000AE060137BFF7A3979AB90FD94E0126F4A
:10761000D712AA1A7F062290FD9AE090FD95600B82
:10762000126F58F990007E74018008126F58F9901B
:10763000007EE41228967F002204F0A3F07DA0FFD4
:1076400012783322E490FEFAF0EF122D8C772701A6
:1076500076770277390376BE04778605767A1277D5
:107660004919771C1A772E1C76751D77391E778F6E
:107670001F000077E7800A027749E5207003027750
:1076800049E4F5207B017AF9797012B8CB7AF9795F
:107690009112B8CB7AF979B212B8CB7AF979D312C0
:1076A000B8CB7AF979F412B8CB7AFA791512B8CB4B
:1076B0007AFA793612B8CB7AFA795702B8CB1277C0
:1076C000F590F903E064406005E014F0800690F95D
:1076D000037443F090F903E0FFB4400890FEFA749D
:1076E00001F08022EFB4410890FEFA7402F0801697
:1076F000EFB4420890FEFA7404F0800AEFB4430637
:1077000090FEFA7408F0E490F904F012780D600627
:1077100012894B1278291289A240A6227A8479D242
:10772000127820744380641277E87442805D7A8412
:1077300079FE127820744180527BFF7A8579141289
:10774000AA1A90F903744080427520FF7B017AF9F0
:10775000797012B8C07AF9799112B8C07AF979B211
:1077600012B8C07AF979D312B8C07AF979F412B89C
:10777000C07AFA791512B8C07AFA793612B8C07A96
:10778000FA795702B8C01277E87442F002ABD4120B
:1077900077F590F903E064406005E014F08006900E
:1077A000F9037443F090F903E0FFB4400890FEFA47
:1077B0007401F08022EFB4410890FEFA7402F08068
:1077C00016EFB4420890FEFA7404F0800AEFB44356
:1077D0000690FEFA7408F012780D600612894B12BA
:1077E00078291289A240AB227BFF7A8479E812AA19
:1077F0001A90F903227BFF7A8479BD12AA1A90F9B4
:1078000001E090F903F090F9027401F0227D0F7FFE
:1078100001129A2990F904EFF090FEFAE05FF0224D
:107820007BFF12AA1A90F9032212AAB490F90274EB
:1078300004F02290FCE2EFF0A3EDF0A3EBF0A3EA5A
:10784000F0A3E9F0129D07A3F0A3F0A3F090FCE2EF
:10785000E0FE129CEFE060037F012274F22E129C86
:10786000F17401F0E5BB54FE4EF5BB75BC0190FC14
:10787000E9E020E12E90FCE3E0F5BDE5B754F144EA
:1078800002129CCAE5BC20E00D1279CA7003129C5A
:10789000F9129C8D40EE129C8A5005129CD48003F4
:1078A000129D0090FCEEE060030279BB90FCE3E0E7
:1078B00020E003027939129D07129CB5400302793A
:1078C0008C90FCEEE0600302798CEF24FFFFEE3435
:1078D000FFFEEDB50715ECB5061190FCE9E020E0E0
:1078E0000AE5B754F1440AF5B78008E5B754F14406
:1078F00006F5B7129CCCE5BC20E00D1279CA7003E6
:10790000129CF9129C8D40EE129D0F90FCEAE0FE55
:10791000A3E0F5828E83E5BF122896129C8A50055B
:10792000129CD48003129D0090FCEBE004F07006E2
:1079300090FCEAE004F00278B9129D07129CB55061
:107940004B90FCEEE07045129D0F8D828C831228C7
:1079500035F5BEE5B754F14406129CCAE5BC20E0FB
:107960000D1279D47003129CF9129C8D40EE129C7A
:107970008A5005129CD48003129D0090FCEBE00419
:10798000F0700690FCEAE004F002793C90FCE9E03B
:1079900020E028E5B754F1440E129CCAE5BC20E073
:1079A0000D1279D47003129CF9129C8D40EE129C3A
:1079B0008A5005129CD48003129D0090FCE2E012D4
:1079C0009CEFE4F090FCEEE0FF2212B91290FCED87
:1079D000E004F02212B91290FCEDE004F02290FED7
:1079E000F9EDF090FEF8EFF0146027146040146099
:1079F0004A14605424FA606C147003027A88240BD1
:107A00006003027AAE90FCD3128C5990FCD3F0F54F
:107A10008022128C7B90FCD4E0FD5EF59090FCCF30
:107A2000E05F62FD128CC590FCD4F0F5902290FCD2
:107A3000D5128C5990FCD5F0F5A02290FCD6128C72
:107A40005990FCD6F0F5B022128C7B90FCD7E0FD6B
:107A50005EF5F290FCD0E05F62F3128CC590FCD72B
:107A6000F0F5F222128C7B90FCDDE0FD5EF58AEFF2
:107A7000C454F0FF90FCE0E090FCDD128CE1540F68
:107A80006F90FCDDF0F58A22128C7B90FCDEE0FD2D
:107A90005EF5C1EF33333354F8FF90FCE1E090FC26
:107AA000DE128CE1541C6F90FCDEF0F5C122128CCA
:107AB000AB704F90FEF8128CBE500724FE60280277
:107AC0007B6612B4E490FEF8128C4DC083C082E055
:107AD000FE90FEF9E0FDEE6DD082D083F074D32FDE
:107AE000128C51E0F59A22128C7B90FCDFE0FD5E57
:107AF000F59190FCD2E05F6297128CC590FCDF029A
:107B00007B6390FEF8E024FA601B14602514602F5C
:107B100024FC603F2407704E90FCD8128C5990FCD6
:107B2000D8F0F59A2290FCD9128C5990FCD9F0F536
:107B3000932290FCDA128C5990FCDAF0F5952290A1
:107B4000FCDB128CCD90FCCEE090FCDB128CECF0D8
:107B5000F5AD2290FCDF128CCD90FCD2E090FCDFE2
:107B6000128CECF0F59122A3F090FC7AE0FF90FCEF
:107B70007DE0FCA3E090FD60FD7B017AFC7981E46F
:107B8000F0A304F02278817CFC7D017BFF122F7131
:107B9000EF2278817CFC7D017BFF122F71EF227830
:107BA000817CFC7D017BFF122F71EF2290FC81F024
:107BB00090FC7AE0FF90FC7CE0FD7B017AFC79810F
:107BC0002278817CFC7D017BFF122F71EF2290FCDB
:107BD0007CE0FEA3E04EF0A3E0F022E4F0A37412F8
:107BE000F07BFF7A6D797390FBCCE4F0A37412F014
:107BF00022F0A3EDF0A3EBF0A3EAF0A3E9F090FCF0
:107C000096E4F0A3740AF0E4A3F0A3F022FDE0FBF5
:107C1000A3E0FAA3E0F9A3E0FFA3E090FCE7CFF034
:107C2000A3EFF0ED22A3F0A37401F0A3227BFF9059
:107C3000FC79E0FFA3E090FBCCCFF0A3EFF022E0D3
:107C4000FEA3E0FF90FC96E0FCA3E0FDC39FEC9E4A
:107C5000227BFF7A6D79E390FC81E090FBCCF022EF
:107C6000D390FC97E0940090FC96E0940022C3909F
:107C7000FC99E0940390FC98E0940022E0FFA3E0DC
:107C800090FBCECFF0A3EFF02278817CFC7D017BCE
:107C9000FF122F71EF22E054FEFD7B0190FCE7E420
:107CA000F0A322A3E024FDF090FC96E034FFF02244
:107CB00090FCE9EFF090FC93E0FF227BFF7A6F7974
:107CC0000D90FBCCF02290FC7AE0FF90FC7CE0224F
:107CD0007BFF7A6D799A2290FC81E0FF90FC7EE038
:107CE0002290FC81E0FF90FC80E02290FFFF122DAB
:107CF000B8EBF090FFFE122DB8ECF0A3EDF012A857
:107D0000FDE58954FCFE12A8DCE0FB4EF5899000ED
:107D100003122DDCE044C0F58B90FF04E014605AA0
:107D2000147003027DC224026003027E1412A8DCD8
:107D300012A8F6EE54FE7009758C16EEC313EF8090
:107D40005F12A8DC12A8F6EE54FC7010758C2DEFB3
:107D50007802CEC313CE13D8F9027E0312A8DC1228
:107D6000A8F6D394EAEE9415500B758CFC7D161290
:107D7000A913027E03AF03027E0D12A8DCA3E0FE6E
:107D8000EE700C758C0E12A8DCA3A3E0027E03EE4D
:107D900054FE700F758C1D12A8DCA3E0C313A3E082
:107DA00013806012A8DC12A8F6D394EFEE94105062
:107DB0000A758CFE7D1112A913804812A8DCE0FF21
:107DC000804B12A8DCA3E0FEEE700B758C1012A89D
:107DD000DCA3A3E0802DEE54FE700F758C2112A859
:107DE000DCA3E0C313A3E013801912A8DC12A8F6E9
:107DF000D394EFEE94105010758CFE7C007D0F1222
:107E000028CAEF14F58D800C12A8DCE0FF12B6989A
:107E10007F00803CAF8C12A8DCE0FD25E02427F831
:107E2000760008A607AF8DED25E02447F876000818
:107E3000A6077401A805088002C333D8FCF588742E
:107E400010A805088002C333D8FC4289D2A97F015B
:107E5000900004022DB8303304D2AED2BE90FF049D
:107E6000E0146078147003027F4624026003027FEE
:107E7000A5E5FF5407B407004003027FB5907E8458
:107E8000F8282873027E99027EA0027EAA027EB4A0
:107E9000027EBE027EC8027ED2786D7603027F38F3
:107EA000786D7601087684027FA5786D7600087675
:107EB000BC027FA5786D7600087658027FA5786DA4
:107EC0007600087626027FA5786D760008760D028A
:107ED0007FA5786D7600087601027FA5E5FF54073F
:107EE000B407004003027FB5907EEFF828287302A4
:107EF0007F04027F0E027F18027F22027F2B027F07
:107F000034027F3D786D7604087607027FA5786D90
:107F100076010876FD027FA5786D76000876F90275
:107F20007FA5786D7600087676807A786D76000881
:107F300076358071786D76000876158068786D7674
:107F400000087604805FE5FF5407B4070050669090
:107F50007F56F8282873027F6B027F74027F7D02B0
:107F60007F83027F8C027F95027F9E786D76040866
:107F700076898031786D760208763E8028786D7635
:107F8000018016786D76000876878019786D760006
:107F900008763D8010786D76000876198007786D38
:107FA0007600087606786EE61846600908E6161828
:107FB00070F31680F02290FD2F126FAB90FD2F1200
:107FC0006F584A4B70030280F490FD2F126F5812C5
:107FD0006FE120E0030280F4126F55F912281C248F
:107FE000FE700302806514607C14600D147003023F
:107FF00080D2240460030280F490FD35126F58F99A
:1080000012281C601DEA494B601890FD2F126F5812
:10801000F912281CFF90FD35126F58F9126FF312F8
:1080200080F5126F46F9126FF304F07D09FC12908F
:108030003E126F462403F9E43AFA126FF3128100FC
:10804000126F462406F9E43AFA126FF304F07D0B3E
:10805000FC12903E126F461271DF126FF304F07D36
:1080600028FC0280F190FD35126F58F912281C602F
:108070001DEA494B601890FD2F126F58F912281C09
:10808000FF90FD35126F58F9126FF31280F5126FE1
:1080900046F9126FF304F07D09FC12903E126F4610
:1080A0002403F9E43AFA126FF3128100126F4624A6
:1080B00006F9E43AFA126FF304F07D0BFC12903EDD
:1080C000126F461271DF126FF37408F07D297C0184
:1080D000801F126F46F9126FF304F07D0AFC1290B4
:1080E0003E126F461271DF126FF37402F07D317C25
:1080F0000112903E22740EF07D127C0112903E22FD
:108100007403F07D0F7C0112903E2290FEF4EFF09C
:10811000A3EDF090FEF4128C4DE04DF0EF14601BD7
:1081200014602B14602F14603024FA603F146051E7
:10813000240B706790FCD3E0F5802290FEF5E0FF01
:1081400090FCCFE05F42FD90FCD4E0F5902290FCE3
:10815000D5E0F5A022128CFE2290FEF5E0FF90FC07
:10816000D0E05F42F390FCD7E0F5F22290FCDDE036
:10817000FF90FEF5128C63FEEF4E90FCDDF0F58A69
:108180002290FCDEE0FF90FEF5128CD990FCE1E03D
:108190005EFEEF4E90FCDEF0F5C122128CAB702D2E
:1081A00090FEF4128CBE500724FE60110282291248
:1081B000B4E490FEF4E0128C4FE0F59A2290FEF5C4
:1081C000E0FF90FCD2E05F4297128D0C2290FEF40B
:1081D000E024FA601514601914601A24FC602F243E
:1081E00007704690FCD8E0F59A2290FCD9E0F59310
:1081F00022128D052290FCDBE0FF90FEF5E090FC62
:10820000CE128C67FEEF4E90FCDBF0F5AD2290FCB9
:10821000DFE0FF90FEF5E0C454F0FE90FCD2E05E9B
:10822000FEEF4E90FCDFF0F5912290FEF6EFF0A30A
:10823000EDF090FEF6128C4DE0FEEDF4FDEE5DF0FB
:10824000EF14601B14602C14603014603124FA6049
:1082500041146054240B706890FCD3E0F5802290A8
:10826000FCD4E0F59090FEF7E0FF90FCCFE05FF4E7
:1082700052FD2290FCD5E0F5A022128CFE2290FC4B
:10828000D7E0F5F290FEF7E0FF90FCD0E05FF4520B
:10829000F32290FCDDE0FFF58A90FEF7128C63F488
:1082A000FEEF5E90FCDDF02290FCDEE0FFF5C19079
:1082B000FEF7128CD990FCE1128CB790FCDEF02214
:1082C000128CAB702E90FEF6128CBE500724FE600E
:1082D0001102834612B4E490FEF6E0128C4FE0F5F2
:1082E0009A22128D0C90FEF7E0FF90FCD2E05FF432
:1082F00052972290FEF6E024FA601514601914607B
:108300001A24FC602C2407703D90FCD8E0F59A22DA
:1083100090FCD9E0F59322128D052290FCDBE0FF62
:10832000F5AD90FEF7E090FCCE128CB390FCDBF044
:108330002290FCDFE0FFF59190FEF7E090FCD21276
:108340008CB390FCDFF02290FDDB126FAB90FDDA76
:10835000EFF012A88A90FDDEE0703B752243FB7AB5
:1083600000792290FCE7F0A312708012783312712A
:108370001590FDDBB5070C126F58F91270001270E2
:10838000B3803D126F58F91270007405F0A37401A8
:10839000F07D75FF802A12711590FDDBB5070F1275
:1083A0006F58F91270007405F0A37402800D126FFB
:1083B00058F91270007405F0A37403F07D757F0105
:1083C00012783390FD09EFF090FD09E0FF60177B14
:1083D000FF7A3879F690FDDA1270DEE4F0A3EFF060
:1083E00012AA1A7F00221270BEA3F0A3F075220118
:1083F000E522601A90FDDB126F5812702055226042
:108400000812713F70031271461271CE80E2127130
:1084100007700312710E90FD0BE07004A3E0640579
:1084200070CB90FD0DE07004A3E064146022127123
:10843000156F601990FDDB126F58F9E490FCE7F0BE
:10844000A3F0A37402F07D757F011278337F0022C0
:108450007F01220D0A0D0A205B4B4C39375D0D0A56
:108460000D0A000D0A0D0A00557365204B4C393773
:108470004320494F20446566696E650D0A005365C7
:1084800074204164383139782053776974636820E7
:1084900052656769737465720D0A005365742041F3
:1084A000643831397820537769746368205265677E
:1084B000697374657220446F6E650D0A0052656DB4
:1084C0006F746520696E2052554E206D6F64650D86
:1084D0000A0052656D6F74652050617373204348C4
:1084E00041206B65790D0A0052656D6F74652050EF
:1084F00061737320434842206B65790D0A00526511
:108500006D6F7465205061737320434843206B6521
:10851000790D0A0052656D6F746520506173732088
:10852000434844206B65790D0A000280004000102A
:108530000020000100020004000002800040001042
:108540000020000100020004000890FED21272A96F
:1085500090FED2127201E412288490FED2127201AF
:108560001273DC127406900003E412289690000443
:108570007440122896900005E4127345C003C002AF
:10858000C00190FED2127201900006122D331273B8
:1085900048C003C002C00190FED2127201900009CF
:1085A000122D33127348C003C002C00190FED212D4
:1085B000720190000C122D33127348C003C002C028
:1085C0000190FED212720190000F122D33127348E7
:1085D000C003C002C00190FED212720190001212BC
:1085E0002D3390FED2127201900015ED127345C02A
:1085F00003C002C00190FED2127201900016122D2B
:1086000033127348C003C002C00190FED21272013F
:10861000900019122D33127348C003C002C001909C
:10862000FED212720190001C122D3390FED21272F3
:108630000190001FE4F5F0022A52128D47F990FBD9
:10864000ACE0FF04F08F827583007480122896904E
:10865000FBACE0FFC374409FC394025007128D41EE
:10866000F912313890FBADE0FEA3E07803C333CEBE
:1086700033CED8F9F0EE90FBADF0E0FF128D47F964
:1086800090003EEF12289690FBAEE090003F12283B
:108690009690FBAF128D27128D93125F7AE490FBB8
:1086A000B3F0A3F0C390FBB4E0941490FBB3E06488
:1086B0008094805066E0FEA3E0FF2498F58274FB6E
:1086C0003EF583E0FD90FF80F0749B2FF58274FBF4
:1086D0003EF583E0FF90FBB3E0FAA3E0FB2498F5BE
:1086E0008274FB3AF583EFF0749B2BF58274FB3AAE
:1086F000F583EDF0128DCBE0FF90FF80128DBFE08F
:10870000FE128DCBEE128DBFEFF090FBB4E024048F
:10871000F090FBB3E03400F00286A4128D9E22900C
:10872000FE54126FABA3EDF090FE54126F584A4BFB
:10873000700302880190FE54126F58126FE120E01E
:10874000030288011270BE90FD0B126F7E7412122C
:108750006F7974DE126F79740FF01270907D027C65
:108760000112903E1270BE90FE57E0FF90FD0BE4A8
:1087700075F00112296BFC748025F0F58274FF3CC2
:10878000F583EF126F7974FF126F79E4F090FD0BAF
:10879000126F7E7463126F797468126F6074451281
:1087A0006F797458126F797450126F797445126F23
:1087B000797450126F79742D126F797453126F7926
:1087C0007470126F79746C126F607474126F7974B4
:1087D00074126F797465126F797472126F79E4F0A4
:1087E00090FD0B126F7EE4F090FD0B126F7EE4F0B3
:1087F00090FE54126F58F91270907D097C0112900E
:108800003E2290FE16E0FBA3E0FAA3E0F9229000DE
:108810001FE4F5F0122A52900015022835E0FEA35D
:10882000E0FF7C007D051228B890FA8CE0FBA3E005
:10883000FAA3E02FF9EA3EA801FCAD037B017AFF21
:1088400079802290001FE4F5F0122A52900016025F
:108850002D0390FA92E0FFC390FA97E09F7480F89E
:1088600090FA96E06480982290001FE475F001125F
:1088700029B9FEC3E5F022FD7401F0A374FFF0A353
:108880007480F02290FA92E075F005A4FF90FA8CC3
:10889000E0FBA3E0FAA3E02FF9EA35F022EBF0A326
:1088A000EAF0A3E9F022C390FA90E094B890FA8F2E
:1088B000E06480948B227E007F051227F690FA9266
:1088C000E004F0229000040228357F057E0012317A
:1088D00014EF22900019022D0390001FE4F5F0021E
:1088E0002A5274FF90F90CF07B017AF9790C90FD13
:1088F000A0E4F0A304F0227401F0A374F9F0742E44
:10890000A3F0A37401F0A32290FDB1E0FF7401A8CD
:1089100007082275F021EFA4240DF582E5F034F963
:10892000F583E02275F021A42412F582E5F034F9F4
:10893000F583E0227B0190FDA0F0A304F0E4FD7F2D
:10894000942290F904E090F90BF02290F903E09062
:10895000F901F022EF75F021A4240DF974F935F036
:10896000FA7B01227401F0A374F9F0A3744F2290F2
:10897000FDB0E0FFC32290FDB0E004F0227B017A5D
:10898000F97901227401F0A374F9F0A3740DF022B7
:10899000A3F07B017AF9790722A3F07B017AF979B8
:1089A000092290F902E004F0E0D39404227B017ADA
:1089B000F979052290F903E0FF90F901E022C0E087
:1089C000C0F0C083C082C0D075D000C000C001C05C
:1089D00002C003C004C005C006C007308812782F4B
:1089E00012A8E36005782F12A8ED758801028A7C31
:1089F000308912783212A8E36005783212A8ED753A
:108A00008802028A7C308A12783512A8E3600578E1
:108A10003512A8ED758804028A7C308B11783812E3
:108A2000A8E36005783812A8ED758808804E308C70
:108A300011783B12A8E36005783B12A8ED75881009
:108A4000803A308D11783E12A8E36005783E12A876
:108A5000ED7588208026308E11784112A8E36005DC
:108A6000784112A8ED7588408012308F0F7844123B
:108A7000A8E36005784412A8ED758880D007D00679
:108A8000D005D004D003D002D001D000D0D0D08205
:108A9000D083D0F0D0E03290FED81272A990FED8E8
:108AA00012720112281CD394014003D38001C340E9
:108AB0000122127296702C90FED812720190000C56
:108AC000127299701E90FED812720190000F1272ED
:108AD00099701090FED81272019000121272997063
:108AE00002C32290FED8127201127296601390FE99
:108AF000D81272011272E9B40103D38001C340019C
:108B00002290FED812720190000C12729960169099
:108B1000FED812720190000C1272ECB40103D380E3
:108B200001C340012290FED812720190000F127210
:108B300099601690FED812720190000F1272ECB478
:108B40000103D38001C340012290FED8127201902C
:108B50000012127299601690FED8127201900012E3
:108B60001272ECB40103D38001C3400122D32290DE
:108B7000FCEF1272A990FCF5127201C003C002C092
:108B80000190FCF2127201900009122D3390FCF852
:108B9000127201C003C002C00190FCF21272019077
:108BA000000C122D3390FCF5127201EA494B60164D
:108BB00090FCF2127201C003C002C001A312720144
:108BC000900006122D3390FCF8127201EA494B60B6
:108BD0001890FCF2127201C003C002C00190FCF8B0
:108BE000127201900006122D3390FCEF127201C038
:108BF00003C002C001A3127201900019122D33901C
:108C0000FCF5127201EA494B601890FCEF127201F8
:108C1000C003C002C00190FCF51272019000161250
:108C20002D3390FCF8127201EA494B601890FCEF6A
:108C3000127201C003C002C00190FCF812720190D0
:108C40000016122D3322E0FF90FEEBE022E0FF241D
:108C5000D3F582E434FCF58322E0FF90FEF9E0FED8
:108C6000EF6E22E090FCE0C454F0FEE05E22E0FEF5
:108C700090FEEBE0C454F0FDEE4D2290FEF9E0FFD3
:108C8000F4FE22C454F0FEEF4EFFF022C454F0F480
:108C9000FEEF5EF02290FEEBE0540FF0A3E0FC222A
:108CA000E0FEC454F05FFFEE4FF02275A101E5A194
:108CB000640122C454F0FEE05EF4FEEF5E22E0FFA9
:108CC00024FB24FB2290FEF9E0FFED6F22E0FF90F1
:108CD000FEF9E0FEC454F0FD22E033333354F8FED5
:108CE000225FFFED6FFFF090FEF9E0225DFDEF6D7A
:108CF000FFF0EE540F6F22F4FEEF5EF0EE2290FCD8
:108D0000D6E0F5B02290FCDAE0F5952290FCDFE0A9
:108D1000F5912290FBBDE0FCA3E0FDA3E0FEA3E003
:108D2000FF90FBB9E0F8A3E0F9A3E0FAA3E0221278
:108D30002CC690FD19E0FCA3E0FDA3E0FEA3E0FF3C
:108D4000227E007F407D0090FBAFE0FBA3E0FAA312
:108D5000E022EB2FFFEA3EFEE93DFDE83CFC22F974
:108D6000A3E0540F75F004A4F58285F08322EF4B45
:108D7000FFEE4AFEED49FDEC48FC226FFFEA6EFE75
:108D8000E96DFDE86CFC225FFFEA5EFEE95DFDE84F
:108D90005CFC2290FD15C9F0A3EAF0A3E9F07B0189
:108DA0007AFB799822EF6BFFEE6AFEED69FDEC68C5
:108DB000FC2290FD19022CC6122C3390FD1222F0D9
:108DC000749A2BF58274FB3AF5832274992BF58201
:108DD00074FB3AF58322F9123138E490FBACF022AF
:108DE0007862A60308A60208A60190FDC5E0F9A3D3
:108DF000E0FAA3E090FD0FC9126FAC90FD0F126F67
:108E00005812702F12810B90FD0F126F5812702F95
:108E10007B0212698890FD0F126F58F912281CFF0F
:108E2000126FE2FD12822A90FD0F126F58F912287C
:108E30001CFF126FE2FD7B0112698812B1AE7D0842
:108E40007F0612810B7B017F061269881270BE12A9
:108E50007120501FEF25E0FFEE33FE90FD0F126FE3
:108E6000581270647B0112698812710770031271C5
:108E70000E80DCE4FB7D01FF12B0147B02E4FD7F79
:108E80000112B0147BFF7AA67926E4FF12B838905D
:108E9000FE6B74FEF07BA0E4FD12ADD87BFF7A0080
:108EA000794EE4FF12B8277D0102AD1F90FD381204
:108EB0006FAB90FD38126F584A4B7002FF2290FD45
:108EC00038126F58126FE120E0037F00227860763D
:108ED000000876017860E6FE08E6FFC3940FEE9482
:108EE000004003028F69EF64054E606F90FD3812F9
:108EF0006F581270D4C00712703F3402FC126FB961
:108F000004F0D00712903EE522F4604FE522604B5A
:108F100090FD38126F581270D4C00712703F34029F
:108F2000FC90FD3B126F58F9126FF3740FF0D007ED
:108F300012903E90FD38126F581270D4C007127014
:108F40003F3403FC90FD3E126F58F9126FF3740E1C
:108F5000F0D00712903E7861E6FF22786106E618AD
:108F60006003028ED406028ED47BFF7A3A79141203
:108F7000AA1A7F0F2290FEE41272A990FEE41272E8
:108F800001127296602190FEE41272011272E9D30E
:108F90009403401390FEE41272019000091273F8DA
:108FA0001272314D12288490FEE412720190000C6E
:108FB000127299602490FEE412720190000C1272F9
:108FC000ECD39403401390FEE412720190000C1253
:108FD00073F81272314D12288490FEE412720190DF
:108FE000000F127299602490FEE412720190000F3B
:108FF0001272ECD39403401390FEE41272019000BD
:109000000F1273F81272314D12288490FEE412721E
:1090100001900012127299602490FEE41272019085
:1090200000121272ECD39403401390FEE41272010A
:109030009000121273F81272314D1228842290FDA2
:1090400052EFF0A3EC126FA61270F890FD52E030D0
:10905000E02614FD7B017AFD79531270001290FA1C
:10906000127078C00690FD52E0FD90FD55126F58C9
:10907000127055E4A3F0802990FD52E0FD7B017A47
:10908000FD79531270001290FA127078C00690FDAC
:1090900052E0FD90FD55126F58127055A37402F006
:1090A000E4FF127833D0E04F90FD09F090FD09E025
:1090B000602390FD0BA3E0FF12B89C1271319480E5
:1090C00040031271A312713F700312714612716353
:1090D000500302904B90FD09E060191271C390FD9E
:1090E00052E090FBCDF090FD53E0FFA3E0CF127073
:1090F000CC12AA1A90FD09E0FF227402F0A314F02A
:10910000E4FF1278332241FA780041F9040041F972
:109110000B0041F9030041F9010041F9020041FA55
:109120008B0041FE410001650042FD070000025E28
:10913000000041FC250041FC2D0F41FC2E00182FA2
:10914000000000000000000000000000000000001F
:1091500000000000000000000F4F000000000000B1
:1091600000000000000000000006140000000000E5
:10917000004DFCD3000000FF000000000000F0E004
:109180000041FCCF0041FCD00041FCE00041FCE18B
:109190000041FCD20041FCCE00C13241FE6C0043D4
:1091A000FE6D00000041FF0401C13341FC95004108
:1091B000FC930042FA8F000043FA8C01FA9841FABE
:1091C000920041FA910043FBAF01FFC00090FF0005
:1091D000EFF0FBC2A9E58954FC4BF589AF8C786AA6
:1091E000760008A607AF8DE4FCFDFE7866122CBA67
:1091F000EB25E0244712A9247866122C7DC3EF9B4F
:10920000FFEE9AFEED99FDEC98FCC004A90512A9A9
:1092100008242712A924D000122A7FC004C00512F6
:10922000A9082428F9C3E7786B96FF19E71896FE7A
:10923000E4FCFDD001D000EB2FFFEA3EFEED39FD4E
:10924000EC38FC7866122CBA90FF04E014601C1411
:10925000602424027033E47F19FEFDFC7866122C32
:109260007D122A7FE47B207A0180147866122C71AB
:10927000E47B0FFA80097866122C71E47B11FAF90D
:10928000F8122B0A7866122CBAD2A97868E6FE0882
:10929000E6FF2290FD9BEF126FA61270F890FD9BE7
:1092A000E030E02614FD7B017AFD799C12700012FB
:1092B000934A127078C00690FD9BE0FD90FD9D12D0
:1092C0006F58127055E4A3F0802990FD9BE0FD7B60
:1092D000017AFD799C12700012934A127078C006D0
:1092E00090FD9BE0FD90FD9D126F58127055A37488
:1092F00002F0E4FF127833D0E04F90FD09F090FDCA
:1093000009E0602390FD0BA3E0FF12B89C127131BD
:10931000948040031271A312713F700312714612C0
:109320007163500302929D90FD09E0FF6016127177
:10933000C390FD9BE090FBCDF090FD9CE090FBCEB8
:10934000F012AA1A90FD09E0FF2204F0A3F0E4FF56
:109350001278332290FCFB1272A990FD0112720167
:10936000C003C002C00190FCFE12720190000F12F7
:109370002D3390FD04127201C003C002C00190FCA5
:10938000FE127201900012122D3390FD0112720133
:10939000EA494B601690FCFE127201C003C002C085
:1093A00001A3127201900006122D3390FD04127277
:1093B00001EA494B601890FCFE127201C003C00222
:1093C000C00190FD04127201900006122D3390FD31
:1093D00001127201EA494B601890FCFB127201C045
:1093E00003C002C00190FD01127201900016122DFF
:1093F0003390FD04127201EA494B601890FCFB1295
:109400007201C003C002C00190FD041272019000FD
:1094100016122D3322C0E0C0F0C083C082C0D075C8
:10942000D000C000C001C002C003C004C005C00617
:10943000C00790FF02E5BBF0E5BB54FE4401F5BB5D
:10944000E5B230E11F7817129CAB6013781E129CB6
:10945000E870010614FF781BE6FD7817129C9D75D5
:10946000B2028050E5B230E211781BE620E00644FB
:1094700001F675B20175B204803AE5B230E31078B6
:109480001E7600087600781BA6B575B2088025E523
:10949000B230E020781BE6FD30E0197817129CAB63
:1094A000600F781E129CE870010614FF7817129C5A
:1094B0009D75B20190FF02E0F5BBD007D006D00544
:1094C000D004D003D002D001D000D0D0D082D0833D
:1094D000D0F0D0E03290FE4D126FAB90FE4CEFF02A
:1094E00012A88A90FE4D126F58F9E412288490FE5B
:1094F0004D126F58F912700012708012783312708A
:1095000078C00690FE4D126F58F91270001270B3B9
:10951000127833D0E04F90FD09F060127BFF7A386B
:10952000798390FE4CE0126FD712717380561270DF
:10953000BEA3F0A3F0752201E522601A90FE4D1241
:109540006F581270205522600812713F700312711B
:10955000461271CE80E2127107700312710E90FDF7
:109560000BE07004A3E0640570CB90FD0DE0700487
:10957000A3E0641460197BFF7A3879A990FE4CE06F
:10958000FF90FBCCE4F0A3EFF012AA1A7F00227F39
:10959000012290FEDB1272A990FEDB1272011272A0
:1095A00096702C90FEDB12720190000C1272997072
:1095B0001E90FEDB12720190000F127299701090D3
:1095C000FEDB1272019000121272997002D3229087
:1095D000FEDB127201127296601090FEDB127201B5
:1095E0001272E9D394014002D32290FEDB12720181
:1095F00090000C127299601390FEDB1272019000C1
:109600000C1272ECD394014002D32290FEDB127252
:109610000190000F127299601390FEDB127201909C
:10962000000F1272ECD394014002D32290FEDB12A1
:109630007201900012127299601390FEDB12720197
:109640009000121272ECD394014002D322C322C0C4
:10965000E0C0F0C083C082C0D075D000C000C0019F
:10966000C002C003C004C005C006C00790FF01E5EA
:10967000BBF053BBFEE5B230E119129CA9600F129A
:109680009CE670010614FF781AE6FD129C9B75B2E9
:1096900002804AE5B230E211781AE620E006440181
:1096A000F675B20175B2048034E5B230E310781C6F
:1096B0007600087600781AA6B575B208801FE5B264
:1096C00030E01A781AE6FD30E013129CA9600B1204
:1096D0009CE670010614FF129C9B75B20190FF017D
:1096E000E0F5BBD007D006D005D004D003D002D01F
:1096F00001D000D0D0D082D083D0F0D0E03290FE24
:1097000070EBF0A3EAF0A3E9F0A3EDF0FF90FBAE5D
:10971000E02FF090FBADE03400F090FE73E0FF70BE
:10972000030297A490FBACE0FEC374409EFEC39F6F
:109730005004AF06800590FE73E0FF90FBB2EFF09F
:109740007E00128D47F990FBACE0FD7C00E92DF91D
:10975000EC3AA801FCAD0390FE70128D4AF9122775
:10976000F690FBB2E0FF90FBACE02FF090FE71E4CE
:109770008FF012295590FE73E0FF90FBB2E0FEC31C
:10978000EF9E90FE73F090FBACE0C39440408B9052
:10979000FBAF128D27128D93125F7A128D41128DBD
:1097A000D602971A2290FD78126FABA3EDF012A7A4
:1097B000E290FD78126F581270D490FD7C126F58B1
:1097C0001270887407F07D1D12929390FD09EFF0DE
:1097D00060127BFF7A38790E90FD7BE0126FD71212
:1097E000717380581270BEA3F0A3F0F522752201A8
:1097F000E522601A90FD7C126F581270205522608D
:109800000812713F70031271461271CE80E212711C
:1098100007700312710E90FD0BE07004A3E0640565
:1098200070CB90FD0DE07004A3E0641460197BFF21
:109830007A38793590FD7BE0FF90FBCCE4F0A3EF24
:10984000F012AA1A7F00227F012290FE2CEEF0A3D4
:10985000EFF0A3EDF090FF04E014600F1460142407
:109860000270507F007ED07D02800E7F807EA97DB9
:109870000380067FB07E1E7D047C00E5FF5407F95F
:10988000F8122BBCE47B20FAF9F812AC5CC006C0DD
:109890000790FE2CE0FEA3E0FBAA06E4F9F8D0074F
:1098A000D00612AC5CC3E49F90FE30F074049E902E
:1098B000FE2FF043878075985090FE2FE0F5BAA3F5
:1098C000E0F5AA75A101E5A1B4010512B39B8003DF
:1098D0007595037E007F147D007B017AFC79BA12B6
:1098E000313890FE2EE06002D2AC22C0E0C0F0C061
:1098F00083C082C0D075D000C000C001C002C003C8
:10990000C004C005C006C007E5F555F6F5233018BC
:1099100011784F12B3426005784F12B34C75F601BF
:10992000804E301911785212B3426005785212B34A
:109930004C75F602803A301A11785512B342600520
:10994000785512B34C75F6048026301B11785812E6
:10995000B3426005785812B34C75F6088012301C7B
:109960000F785B12B3426005785B12B34C75F6104A
:10997000D007D006D005D004D003D002D001D0004B
:10998000D0D0D082D083D0F0D0E03290FE7E126F63
:10999000AB90FE7E126F58F9ED12288490FE7E1275
:1099A0006F58F9900001E4122896126F927D05120B
:1099B000929390FD09E07024E522602090FE7E12D3
:1099C0006F58126FD37BFF7A37799112AA1A90FEE3
:1099D0007E126F581270AA44401228847522089093
:1099E000FE7E126F58F912281C126F967D07129294
:1099F0009390FE7E126F58126F917D071292939092
:109A0000FD09E0702330132090FE7E126F58126F14
:109A1000D37BFF7A3779B012AA1A90FE7E126F5864
:109A20001270AA448012288422AB05AA07EA1460A7
:109A30001C14601E14602014602224FA6023146039
:109A400025146027240C703EE5805BFF22E5905BC7
:109A5000FF22E5A05BFF22E5B05BFF22E5F25BFFA2
:109A600022E58A5BFF22E5C15BFF22E58F5470FA95
:109A7000758F7090FCD1E591F0E4F58FE04591F0A1
:109A80008A8FE05BFF2275A101E5A1B40113EA24EE
:109A9000FB24FB5002802CAF0212B4E4E59A5BFF7A
:109AA00022EA24FA600F1460111460132403701367
:109AB000E59A5BFF22E5935BFF22E5955BFF22E5DC
:109AC000AD5BFF2290FEDE1272A990FEDE127201E3
:109AD000127296601590FEDE1272011272E9FF6436
:109AE000036007EFD3940140012290FEDE12720161
:109AF00090000C127299601890FEDE1272019000B4
:109B00000C1272ECFF64036007EFD3940140012252
:109B100090FEDE12720190000F127299601890FE92
:109B2000DE12720190000F1272ECFF64036007EF07
:109B3000D3940140012290FEDE12720190001212B5
:109B40007299601890FEDE1272019000121272EC8F
:109B5000FF64036007EFD39401400122D322303326
:109B600004D2AED2BE90FF04E014603014605624DC
:109B7000027079E5FF540714601014601314601626
:109B800024037070786C767E8062786C7637805CA7
:109B9000786C76138056786C76018050E5FF540718
:109BA00014601014601314601624037047786C76E8
:109BB000A98039786C764C8033786C761E802D784D
:109BC0006C76078027E5FF540714601014601314A7
:109BD00060162403701E786C76C08010786C7658FE
:109BE000800A786C76248004786C760A786CE6605B
:109BF000031680F82290FE7BEB125C6190FE7B12D4
:109C00005B9F125D296003029C8790FE42F0A37463
:109C100004F090FE7B125B9F125EA1FF125C1B1290
:109C20005CFA50527480125F1654E06460701F74C6
:109C300081125F1664037033125C832482125DE12B
:109C4000640C70277483125DE070207F012290FE07
:109C50007B125B9F90FE43E02480125C2E8F82F586
:109C600083122835125F2B125C2FF0125C9370A2C6
:109C7000125CC6029C1290FE7B125B9F125EA112C8
:109C80005CE140037F00227F002275BC01C390FC91
:109C9000EDE094A890FCECE0946122781408E6FAD8
:109CA00008E6F5828A83022DB67814860308E6FA60
:109CB00008E64A4B2290FCE7E0FEA3E0FF90FCEAB6
:109CC000E0FCA3E0FDC39FEC9E22F5B7E490FCEC22
:109CD000F0A3F022E5BC540690FCEEF022ED540116
:109CE000C4333354C022781C0806E61886062224A2
:109CF000F2F582E434FEF5832290FCECE004F022DD
:109D000090FCEE7403F022E490FCEAF0A3F02290C1
:109D1000FCE4E0FBA3E0FAA3E0F92290FD5AEFF0A7
:109D2000A3EC127BF190FC93E0FF90FD5A7AFD7951
:109D30005B127C967402F0A314F012783390FC94BA
:109D4000EFF0E0FEC00690FD5AE090FD5D127C0D44
:109D500030E0047F0080027F02127CB0127833D0A2
:109D6000E04F90FC94F0602390FC97E0FF12B89CC9
:109D7000127C604003127CA390FC99E004F0700612
:109D800090FC98E004F0127C6E409A90FC94E060A5
:109D900014127CBB90FD5AE090FBCDF090FD5B125D
:109DA0007C7C12AA1A90FC94E0FF2290FDA2EF1294
:109DB0007BF190FC93E0FF90FDA27AFD79A3127CE9
:109DC0009604F0A3F012783390FC94EFF0E0FEC01C
:109DD0000690FDA2E090FDA4127C0D30E0047F000F
:109DE00080027F02127CB0127833D0E04F90FC9456
:109DF000F0602390FC97E0FF12B89C127C60400357
:109E0000127CA390FC99E004F0700690FC98E004AA
:109E1000F0127C6E409C90FC94E0FF6016127CBBBC
:109E200090FDA2E090FBCDF090FDA3E090FBCEF082
:109E300012AA1A90FC94E0FF2290FE81126FAB9060
:109E4000FE81126F58126FE130E51F30E60820E7FF
:109E50004C127008802690FE81126F581270071203
:109E60009EBA126F58127007802B90FE81126F58A5
:109E7000126FE130E60D20E724127015F07B067DAD
:109E800006801790FE81126F58127014129EBA123B
:109E90006F58127014F07B047D0A12AB8F90FE8114
:109EA000126F58126F917D0612929390FE81126F7D
:109EB00058126FD31270EA02AA1AF07B057D0A12BB
:109EC000AB8F90FE8122787FE4F6D8FD7581700219
:109ED0009F0D023B89E493A3F8E493A34003F6802B
:109EE00001F208DFF48029E493A3F85407240CC896
:109EF000C333C4540F4420C8834004F45680014641
:109F0000F6DFE4800B0102040810204080909106E7
:109F1000E47E019360BCA3FF543F30E509541FFE6B
:109F2000E493A360010ECF54C025E060A840B8E4DC
:109F300093A3FAE493A3F8E493A3C8C582C8CAC55F
:109F400083CAF0A3C8C582C8CAC583CADFE9DEE7F1
:109F500080BE90FEE71272A990FEE71272011272A3
:109F600096601390FEE71272019000091273FF12BF
:109F700072314D12288490FEE712720190000C128B
:109F80007299601390FEE712720190000C1273FF39
:109F90001272314D12288490FEE712720190000F68
:109FA000127299601390FEE712720190000F127303
:109FB000FF1272314D12288490FEE7127201900058
:109FC00012127299601390FEE71272019000121241
:109FD00073FF1272314D1228842290FECF126FABA4
:109FE00090FECF126F584A4B7002C32290FECF12E0
:109FF0006F58126FE120E002C322D390FD08E09475
:10A000002090FD07E064809480401C90FECF126F8A
:10A0100058126FD37BFF7A3A794A12AA1AE490FD5C
:10A0200007F0A3F07865F67865E6603290FECF120F
:10A030006F58F9126FB404F07D05FC12903E301198
:10A040000F7865E6600116E490FD07F0A3F0D322D7
:10A0500090FD08E004F0700690FD07E004F0C322D4
:10A0600090FEE11272A990FEE112720112729660E6
:10A070001190FEE11272019000091272F220E402C6
:10A08000C32290FEE112720190000C1272996011CD
:10A0900090FEE112720190000C1272F220E402C3F1
:10A0A0002290FEE112720190000F127299601190DD
:10A0B000FEE112720190000F1272F220E402C3223C
:10A0C00090FEE1127201900012127299601190FEDE
:10A0D000E11272019000121272F220E402C322D344
:10A0E0002290FE93126FAB90FE93126F58126FE1A5
:10A0F00030E63475220812281C126F967D051292E4
:10A100009390FE93126F58126FE130E7057522A00D
:10A11000800A75229490FE93126F58F912281C122F
:10A120006F967D0612929390FE93126F58F9129ECD
:10A130003990FE93126F58F912A97F90FE93126F17
:10A1400058126FE130E708127008F07B03800B9023
:10A15000FE93126F58127007F0FB7D0712AB8F222F
:10A1600090FF04E014602714604424027067E5FF48
:10A17000540714600D14601024027061786C7645E9
:10A180008053786C761B804D786C76058047E5FFB0
:10A19000540714600D14601024027041786C765FCF
:10A1A0008033786C7628802D786C760C8027E5FFDC
:10A1B00054071460101460131460162403701E7882
:10A1C0006C766D8010786C762F800A786C760F80B4
:10A1D00004E4786CF6786CE660031680F82290FE52
:10A1E000CC126FABED12288490FECC126F58127017
:10A1F000D490FD58126FC97402F07D007C04129057
:10A200003E90FD09EFF090FECC601C126F58126F6B
:10A21000D37BFF7A3979CF12AA1A90FECC126F58ED
:10A22000F9900001E4802E126F58126FD390FF80D6
:10A230001270C990FF81E0FF90FBD0E4F0A3EFF033
:10A240007BFF7A3979F112AA1A90FECC126F58F975
:10A2500090000174011228962290FE44126FABA365
:10A26000EDF012A7E290FE44126F58126F917D0933
:10A270001292933011037F012290FE47E0FF12A853
:10A280008AE4F522FB90FCE7126FBF1271B01278DE
:10A290003390FCE7126F9A12714F127833E4F52273
:10A2A000FB90FCE7126F9DA3F07DA0FF12783312A4
:10A2B0007078C00690FCE7126FBC0412715A1278D5
:10A2C00033D0E04F90FD09F070037F02227F00221F
:10A2D000C0E0C0F0C083C082C0D075D000C000C054
:10A2E00001C002C003C004C005C006C007C2327569
:10A2F000A101E5A164017019F5A612B6EE602AE588
:10A30000A530E6047F0180027F0012B6FDADA78074
:10A310001512B6EE6013E5A530E6047F0180027FDA
:10A320000012B6FD7D10122DB643A580D007D006D1
:10A33000D005D004D003D002D001D000D0D0D0823C
:10A34000D083D0F0D0E03290FE25EDF090FE22EBED
:10A35000125C61125F35C39401405F90FE26E0FFFE
:10A3600090FE42E4F0A3EFF090FE22125B9F125E9B
:10A37000A12480FFE433FE125C1BC3125D4F502307
:10A38000125C0DFE54E0FF90FE25E0B50703AF051B
:10A3900022EE125F2B125C2FF0125C9370CA125CDB
:10A3A000C680C590FE22125B9F125EA12480FFE44E
:10A3B00033FE125D4D40037F00227F002290FE5C41
:10A3C000126FABA3EDF090FE5C126F584A4B6051D8
:10A3D00090FE5C126F58126FE130E045E490FF8010
:10A3E000F0126FE904F0FDFC12903E90FF8074FFC4
:10A3F00012710090FE5C126F58126FE812A4227F57
:10A400000A12B89C90FF807405F090FE5FE090FF08
:10A4100081F0E4A3F090FE5C126F58126FE812A472
:10A4200022227403F07D207C0112903E2290FD4197
:10A43000126FABA3EDF090FD41126F584A4B60577D
:10A4400090FD41126F58126FE130E04B12281C7AD8
:10A45000FD7944126FF004F0FDFC12903E90FD4631
:10A46000E0FE602090FD41126F58F912281CFF9009
:10A47000FD47126F58F9EEFD126FF3EDF07D007C91
:10A480000512903E90FD41126F58F912281CFF9062
:10A49000FD45E0FD12A5C42290FDA912889D1288F9
:10A4A0004CC003C002C00190FDA912880512881794
:10A4B000FD90FD8A7401F0A374FDF0A374ACF0D09C
:10A4C00001D002D00312AB49EF7002FF2290FDA928
:10A4D000128805128817FF7B017AFD79AE12A4FF5E
:10A4E000EF7002FF2290FDAEE0FEA3E0FF90FDAC16
:10A4F000E0B50608A3E0B507037F01227F002290A4
:10A50000FE51126FAB90FE50EFF012A88A90FE51F0
:10A51000126F58F9740812288490FE51126F58F97E
:10A52000127000127080127833127078C00690FE9C
:10A5300051126F58F912700074021270B51278330C
:10A54000D0E04F90FD09F060167BFF7A3879CF900C
:10A55000FE50E0126FD71270C612AA1A7F00227F37
:10A56000012290FDEC126FAB90FDEC126F584A4B3C
:10A570007002FF2290FDEC126F58126FE120E00391
:10A580007F0022126FB404F07D507C0212903EE5F1
:10A5900022F46024E522602090FDEC126F581270C6
:10A5A000D490FDEF126F58F9126FF37409F07D50DB
:10A5B0007C0212903E7F05227BFF7A3A792C12AA08
:10A5C0001A7F002290FE60EFF0ED1270FF90FE60A7
:10A5D000E0126FB704F07D06FC12903EEF7004E5C8
:10A5E0002260187F0A12B89C90FE63E004F07006A7
:10A5F00090FE62E004F012718740D2127187401021
:10A600007BFF7A3A796E90FE60E0126FD712AA1A39
:10A6100090FE60E0FF7B017AFE7961126FF304F037
:10A620007D06FC02903E90FEF0EEF0A3EFF0ED30E0
:10A63000E00A785F06E618703506803290FEF0E09A
:10A640007002A3E0703D786FA6B5ED540E785E768B
:10A650000008F618E6FE08E67807C333CE33CED8F6
:10A66000F9FF786FE6FDEE785EF6EF4D08F678625A
:10A67000860308E6FA08E6F9785EE6FE08E6127058
:10A6800028F5B42290FEEFEDF090FEEDEEF0A3EF92
:10A69000F0C3EE9402504674806480700374FFF43B
:10A6A000703B30AF04D2318002C231C2AF90FEEEB7
:10A6B000E0240090FEEDE034EEF5F9A3E0F5FA7841
:10A6C000C07CFF79C07E0012B8EC90FEEFE078709D
:10A6D000F67B01797012FFC0303102D2AF2290FEBA
:10A6E00078EB125C6190FE78125B9FEA494B604602
:10A6F00090FE78125BED125D3D7A5179637E017FA9
:10A70000001227F690FC9D74FFF0A37451F0A3741F
:10A7100063F0E4A3F090FE78125B9F12028090FE3B
:10A7200078125BED125F0C44011228844402122857
:10A730008454FB1228842290FE3B12B386A3ECF0D3
:10A74000A3EDF0E4FDFCD390FE3FE09DEC6480F8C7
:10A7500090FE3EE0648098402F12B3FDEFF460F964
:10A7600012B38F8D828C83EF122896EFB40A12ED0C
:10A770001D70011C12B38F8D828C83E41228968089
:10A78000070DBD00010C80BEAE04AF052290FE583F
:10A79000126FABA3EDF090FE58126F584A4B604118
:10A7A00090FE58126F58126FE130E03512281CFFEE
:10A7B0007D0412A5C490FE5BE0F52290FE58126F56
:10A7C00058F912281C126FB804F07D007C05129015
:10A7D0003E90FE58126F58F912281CFF7D0312A5F7
:10A7E000C42290FE67EDF090FE64126FAB126F9280
:10A7F0007D0712929390FE64126F58126FE130E75A
:10A800001490FE67E05403FFE52254036F6026E5D1
:10A810002254FC801290FE67E05401FFE5225401AF
:10A820006F6012E52254FE4FF52212281C126F961B
:10A830007D0712929322C0E0C083C082C0D075D041
:10A8400000C004C005C007E59830E02F90FCCCE0C4
:10A85000FF2401FDE433FCA3E06D7001EC6019748A
:10A86000BA2FF582E434FCF583E599F090FCCCE056
:10A8700004F0E0B41202E4F05398FED007D005D003
:10A8800004D0D0D082D083D0E03290FEFFEFF0121F
:10A8900070BE127120504274047E00A80708800523
:10A8A000C333CE33CED8F9FF90FEFFE0FDEF5D90CD
:10A8B000FD0C600E127195126F5812706412810BAC
:10A8C000800C127195126F5812706412822A1271E4
:10A8D00007700312710E02A89202B4BE851283851E
:10A8E000138222860308E6FA08E64A4B2208E6FAB3
:10A8F00008E6F9022DB2A3E0FEA3E0FF2290FFFFDD
:10A90000122DB8EFF0C2A922AA06AB0790FF00E013
:10A9100025E0227C001228CAEF22F8A60308A6022E
:10A9200008A60122F8E6FE08E6FFE4FCFD2290FE00
:10A930003112B386A3ECF0A3EDF0E4FFFE75A101A4
:10A94000E5A1B4010512B39B8003759503D390FE76
:10A9500035E09FEE6480F890FE34E0648098401EFD
:10A9600090FE3112B3928F828E83122835F599E5CD
:10A970009830E1FB5398FD0FBF00010E80CF22906D
:10A98000FE87126FAB90FE87126F58126FE130E4B2
:10A990000830E61C127015800F90FE87126F581257
:10A9A0006FE130E60B127008F07B077D0612AB8F6B
:10A9B00090FE87126F58126F917D0612929390FE4F
:10A9C00087126F58126FD31270EA02AA1A90FF040E
:10A9D000E014601314602624027036E5FF540770FB
:10A9E00038786C760D802AE5FF54071460090470EE
:10A9F00028786C7615801A786C76038014E5FF54FD
:10AA000007146009047012786C761A8004786C76EA
:10AA100005786CE660031680F82290FBC912B386B5
:10AA200090FBF47401F0A374FBF0A374CCF090FBE2
:10AA3000C9E0F9A3E0FAA3E090FE1CC912B3879025
:10AA4000FBF4E0F9A3E0FAA3E090FE1FC912B3877C
:10AA500012B3A812AAFF12B3A812B7B2AC06AD0780
:10AA600012B3A812A92E2290FE741231917810EC24
:10AA70004D4E4F70047CA57DA5C3EC13FCED13FD7A
:10AA8000EE13FEEF13FF5010EC64CCFCED644CFDB4
:10AA9000EE644EFEEF64CEFFD8DF90FE74122CC63B
:10AAA000EE547FFE2290FE74EEF0EFA3F0A374A5A7
:10AAB000F0A3F022E490FEFBF0F07AFE79FB12891D
:10AAC000341292937B017AFE79FB1288EE12AAF877
:10AAD0007F0112B8A812897D1288EEE412AAF8123A
:10AAE000897D1288EEFD7F941292937F0212764444
:10AAF000E490FA8BF0D20D22FD7F94129293229073
:10AB0000FE1CE0FFA3E0FEA3E0CF90FC54F0A3EE18
:10AB1000F0A3EFF090FE1FE0CBF0A3E0CAF0A3E0BB
:10AB2000C9F07F2290FC57AD82AC8312281C8D8225
:10AB30008C83F0A309E970010ADFEC90FE1FE0FBB3
:10AB4000A3E0FAA3E0F902636690FD86126FABA35F
:10AB5000EDF012A7E290FD86126F581270D490FDAE
:10AB60008A126F581270887402F07D2212929390AC
:10AB7000FD09EFF060167BFF7A38795B90FD89E084
:10AB8000126FD71270C612AA1A7F00227F0122907C
:10AB9000FE29EBF090FE27EFF0A3EDF0EF126F959A
:10ABA00012929390FE2AE07002A3E0600D1271B839
:10ABB0008002C333D8FC4222800C1271B88002C3D9
:10ABC00033D8FCF4522290FE27E0FFA3E0FD126F81
:10ABD000970292931289B46F603DEFB440047E01F6
:10ABE000801AEFB441047E028012EFB442047E0466
:10ABF000800AEFB443047E088002E4FEE490F90486
:10AC0000F07D0F7F01129A2990F904EFF05EFE604B
:10AC10000612894B12AAB42290FE48126FABA3ED24
:10AC2000F012A7E290FE48126F58126F917D0F123A
:10AC3000929390FD09EFF0601D7BFF7A3779E890E1
:10AC4000FE4BE0126FD790FD09E090FBCE126FDA59
:10AC500012AA1A7F0022A217E433FF22C2D5E830DD
:10AC6000E70FB2D5E4C39BFBE49AFAE499F9E498C0
:10AC7000F8EC30E717B2D512AC92122B0AE4C39B62
:10AC8000FBE49AFAE499F9E498F88003122B0A306D
:10AC9000D50DE4C39FFFE49EFEE49DFDE49CFC22F1
:10ACA0001289B4FD6F6038EDB443047E08801AED5C
:10ACB000B442047E048012EDB441047E02800AEDA9
:10ACC000B440047E018002E4FE7D0F7F01129A29C8
:10ACD00090F904EFF05EFE700612894B12AAB422BE
:10ACE00090FD4A126FAB90FD4A126F584A4B7003A9
:10ACF0007F012290FD4A126F58126FE120E0037F1E
:10AD0000012212281C04FF90FD4D126F58F9A31266
:10AD1000709D7D007C0712903E90FD09EFF022901F
:10AD2000FFFF122DB8EDF012B33312B3558002C3FA
:10AD300033D8FC12B33BF0E0FF42F312B33BA3E085
:10AD40006005EF42F4800712B33BE0F452F412B313
:10AD50003BE0F5F6D2A842F5900002022DB8E4904F
:10AD6000FEFCF0F07AFE79FC1289341292937B019A
:10AD70007AFE79FC1288EEFD7F941292937F011285
:10AD8000B8A812897D1288EEE4FD7F941292931286
:10AD9000897D1288EEFD7F9402929390FB98122C8D
:10ADA000D26745230190FB9C122CD2EFCDAB89904A
:10ADB000FBA0122CD298BADCFE90FBA4122CD2106D
:10ADC00032547690FBA8122CD2C3D2E1F0128D41FE
:10ADD000128DD6A3F0A3F02290FE6AEBF0EF601480
:10ADE000D2BAED6006D2B6D2B78004D2B4D2B5439F
:10ADF000BB048012D2B9ED6006D2B2D2B38004D2C5
:10AE0000B0D2B143BB0212B50A90FE6AE0F5B3A31B
:10AE1000E0F5B62290FE3612B386E4A3F0A3F090DC
:10AE2000FE3612B392A3E0FEA3E0F5828E831228D1
:10AE300035FF601312B75890FE3AE004F070E090CE
:10AE4000FE39E004F080D890FE39E0FEA3E0FF2256
:10AE500090FD1DEB125C6190FD1D125BED125D3DDE
:10AE60007A5279697E007F031227F690FD20125BEB
:10AE70009F740312288490FD23125BED125D3D7ACE
:10AE800052796C7E007F030227F690FD26EB125C60
:10AE90006190FD26125BED125D3D7A5279767E005F
:10AEA0007F091227F690FD29125B9F7409122884EE
:10AEB00090FD2C125BED125D3D7A52797F7E007F12
:10AEC000030227F690FE8D126FAB90FE8D126F5825
:10AED000126FE130E60B127008F07B057D0612ABB5
:10AEE0008F90FE8D126F58126F917D061292939083
:10AEF000FE8D126F58126FD31270EA02AA1A75A152
:10AF000001E5A1B4011BEF24FE600C14600E2403C4
:10AF1000702375A49C801E75A4DC801975A4FC8028
:10AF20001443F580EF24FE60092402700875A4B86C
:10AF3000800375A4F8D2BD22AE07E4FF12B424BF8B
:10AF4000010AEE7007EDB41003D20922E4FF12B437
:10AF500024EF700AEE7007EDB41003D20922E4FF6B
:10AF600012B424BF8009EE7006EDB41002D209229B
:10AF700090FEC6126FAB12A88A90FEC6126F58F9E7
:10AF8000744112288490FEC6126F58F91270001294
:10AF9000708012783390FEC6126F58F912700074E8
:10AFA000021270B502783390FEC9126FAB12A88AF4
:10AFB00090FEC9126F58F9742012288490FEC912AD
:10AFC0006F58F912700012708012783390FEC91217
:10AFD0006F58F912700074141270B502783390FD36
:10AFE000F2126FAB90FDF2126F584A4B602590FD44
:10AFF000F2126F58126FE130E01912281C04FF9012
:10B00000FDF5126F58F9126FF3740FF07D007C029A
:10B0100012903E22EF6019D2BAED6006D2B6D2B7D6
:10B020008004D2B4D2B543BB04E490FEF3F08017A1
:10B03000D2B9ED6006D2B2D2B38004D2B0D2B1435D
:10B04000BB02E490FEF2F002B2B490FDE0126FABEE
:10B0500090FDE0126F584A4B602490FDE0126F584B
:10B06000126FE130E01812281CFF90FDE3126F58B8
:10B07000F9126FF37402F07D077C0112903E22906A
:10B08000FDE6126FAB90FDE6126F584A4B602490BC
:10B09000FDE6126F58126FE130E01812281CFF9085
:10B0A000FDE9126F58F9126FF37403F07D0C7C0107
:10B0B00012903E2290FDF8126FAB90FDF8126F587F
:10B0C0004A4B602490FDF8126F58126FE130E0187F
:10B0D00012281CFF90FDFB126F58F9126FF37408D1
:10B0E000F07D207C0112903E22E490FEFDF0F07B8A
:10B0F000017AFE79FD1289361292937B017AFE79EC
:10B10000FD1288EEFD7F941292937F0112B8A87F02
:10B1100002127644E490FA8BF0D20D2290FE961241
:10B120006FAB90FE96126F58126F917D071292933B
:10B1300090FE96126F58126FE130E708A216821740
:10B1400082138006A21682178211E433FF2290FD3B
:10B15000FE1272A990FDFEE0F9A3E0FAA3E090FCD4
:10B160002FC91272AA90FE01E0F9A3E0FAA3E090C1
:10B17000FDC5C91272AA90FDFE127201028DE07423
:10B18000806480700374FFF4702330AF04D2318088
:10B1900002C231C2AF75F9EEE4F5FA78807CFF792E
:10B1A00080FE12B8EC12FF80303102D2AF2290FD47
:10B1B0000F126F58F912281CFF126FE2FD12822A3B
:10B1C000129B5E90FD0F126F58F912281CFF126F30
:10B1D000E2FD12810B7F0402B89C90FE90126FABCF
:10B1E00090FE90126F58126FE130E708127015F060
:10B1F0007B03800C90FE90126F58127014F07B014C
:10B200007D0712AB8F2290FD71126FAB90FD711212
:10B210006F58F912A7E290FD71126F58F912281CAD
:10B22000FF90FD75126F581270887408F07D15023A
:10B23000929390FD7F126FAB90FD7F126F58F912C1
:10B24000A7E290FD7F126F58F912281CFF90FD8332
:10B25000126F581270887405F07D1002929390FE60
:10B2600084126FABED90FE84600A126F581270AAC0
:10B2700044208008126F581270AA54DF122884905C
:10B28000FE84126F58F9029E3990FE8A126FABED60
:10B2900090FE8A600A126F581270AA441080081239
:10B2A0006F581270AA54EF12288490FE8A126F58B9
:10B2B000F902A97FEF600543BB01800353BBFEED9C
:10B2C000B4020CEB5403C454F0FF129CDD800C124A
:10B2D0009CDD4480FFEB5403C454F04FF5B722903B
:10B2E000FEBD126FAB90FEBD126F58F912A7E2902F
:10B2F000FEBD126F58126F917D0F129293E52230AE
:10B30000E1047F0180027F002290FD8D126FAB90DF
:10B31000FD8D126F58F912A7E290FD8D126F581231
:10B3200070D490FD91126F581270887408F07D25CA
:10B3300002929390FFFF122DB8EFF08512838513D0
:10B340008222860308E6FA08E64A4B2208E6FA0853
:10B35000E6F9022DB2E0FF7401A807082290FEFE74
:10B36000EDF012A88A752215126FFA127080127809
:10B37000337B017AFE79FE12700004F0A304F07DA5
:10B38000747F01027833EBF0A3EAF0A3E9F0229096
:10B39000FE3BE0FBA3E0FAA3E0F92275A102439A89
:10B3A00003439C03539BFC227B017AFF798022900C
:10B3B000FEC0126FAB12A88A752218126FFA1270B3
:10B3C0008012783390FEC0126F58F9127000740822
:10B3D0001271D502783390FEC3126FAB12A88A7532
:10B3E0002210126FFA12708012783390FEC3126F1F
:10B3F00058F912700074051271D50278337FFF90EE
:10B40000FCCDE0FE90FCCCE06E601874BA2EF582A4
:10B41000E434FCF583E0FF90FCCDE004F0E0B412EE
:10B4200002E4F02230320CEF70037F862290FE6C33
:10B43000E0FF2275A101E5A1B40107EF04F5A6AF75
:10B44000A722EF7003AFA622AFA722EFB40A0774BA
:10B450000D12B456740A309811A899B8130CC298FA
:10B460003098FDA899C298B811F63099FDC299F5A7
:10B47000992290FDB6EB125C6190FDB6125BED1265
:10B480005D3D7A5279637E007F061227F690FDB902
:10B49000125B9F740602288490FDBCEB125C6190E5
:10B4A000FDBC125BED125D3D7A52796F7E007F0725
:10B4B0001227F690FDBF125B9F740702288412B911
:10B4C0000AE6FF700476178012EFB40106786C76F6
:10B4D000098008EFB4020C786C7602786CE66003A1
:10B4E0001680F822EF24FA6011146012146013140D
:10B4F000601424047013E4F5A12275A1012275A142
:10B50000022275A1032275A10422E5BB54FE4FF56A
:10B51000BBEDB40208129CDE442EF5B122129CDD74
:10B5200044AEF5B175B4FF75B21F43B1012212B933
:10B530000AE6FF7004760C800FEFB40106786C7693
:10B54000048005EFB4020922786CE660031680F8E7
:10B550002290FE9F126FAB90FE9F126F58F912A7B8
:10B56000E290FE9F126F58127007F0E4FB7D080214
:10B57000AB8F90FEA2126FAB90FEA2126F58F91221
:10B58000A7E290FEA2126F58127007F07B077D08A9
:10B5900002AB8F90FEA5126FAB90FEA5126F58F90B
:10B5A00012A7E290FEA5126F58127014F07B077D6F
:10B5B0000802AB8F90FEA8126FAB90FEA8126F58D6
:10B5C000F912A7E290FEA8126F58127007F0E4FB80
:10B5D0007D0F02AB8F90FEB1126FAB90FEB1126F78
:10B5E00058F912A7E290FEB1126F58127007F0E4FA
:10B5F000FB7D0E02AB8F90FEB7126FAB90FEB712C1
:10B600006F58F912A7E290FEB7126F58127007F048
:10B610007B047D0F02AB8F90FEBA126FAB90FEBA27
:10B62000126F58F912A7E290FEBA126F58127014F6
:10B63000F07B047D0F02AB8F90FE9C126FAB90FEEF
:10B640009C126F58F912A7E290FE9C126F5812706C
:10B6500014F0FB7D0802AB8F90FEAB126FAB90FE37
:10B66000AB126F58F912A7E290FEAB126F5812702E
:10B6700014F0FB7D0F02AB8F90FEB4126FAB90FE07
:10B68000B4126F58F912A7E290FEB4126F581270FC
:10B6900014F0FB7D0E02AB8F12A8FD12A8DCE0FFB8
:10B6A0007410A807088002C333D8FCF45289D2A9C9
:10B6B000900001022DB812A88A752240126FFA126A
:10B6C0007080127833126FFA041270B5127833AFAB
:10B6D000222212B90AE6FF700476098008EFB4014D
:10B6E0000C786C7602786CE660031680F82290FE87
:10B6F0006DE0FBA3E0FAA3E0F9EA494B2290FE6D6E
:10B70000A3E0FAA3E0F5828A8322EF6007D23375C3
:10B7100086808002C233D2AFE5FFB430037F0122BE
:10B7200075FF307F002212B33312B3558002C3334A
:10B73000D8FC12B33BF0E055F2FF900001022DB8A7
:10B7400012281CFF90FD6D126F58F9A3E0FD1270D6
:10B7500089EDF07D8002929390FF03EFF07B017AF8
:10B76000FF79037D017C0012A92E90FF03E0FF22E8
:10B77000C3EE940240037FFF2274002FF58274EE23
:10B780003EF583E493FF2212281C04FF90FDD112A2
:10B790006F581270887408F07D4102929312B3338F
:10B7A00012B3558002C333D8FCF452F59000010265
:10B7B0002DB8E4FFFE12281C600C0FEF70010E097B
:10B7C000E970F20A80EF2210340B12B8F7BF0D02B5
:10B7D0007F0A02B44B90FF06E0FF22EFC3940940BA
:10B7E00005EF940E4004EFB42003D38001C32290F0
:10B7F000FD0F126F5812702F12810B7D02E4FF02B1
:10B80000B50AC003C002C00190FE07127201900089
:10B810001C122D3322E4FDFF12B50A90FD0F126FAA
:10B820005812702F02822AEF75F003A4244FF8A655
:10B830000308A60208A60122EF75F003A42414F859
:10B84000A60308A60208A60122786C7664786CE646
:10B85000166005127E5680F522126F927D071292B5
:10B8600093A215E433FF22126F927D08129293A2E5
:10B8700016E433FF22126F927D40129293A210E4DD
:10B8800033FF22126FE230E6047F0180027F002244
:10B89000AE071FEE6005129B5E80F522AE071FEE1D
:10B8A0006005127E5680F522AE071FEE600512B8C5
:10B8B0004980F52290FE6DEBF0A3EAF0A3E9F022B7
:10B8C000E924041272314420022884E9240412720B
:10B8D0003154DF022884EF75F003A4242F12A91A33
:10B8E00022EF75F003A4243B12A91A227D017BFFED
:10B8F0007AFF7F400227F63098FDAF99C2987E000C
:10B900002290FE99126FAB7F0022E5FF5407786CFE
:10B91000F622303304D2AED2BE2290FF06EFF0D230
:10B92000342290FF04EFF022D20822FFFFFFFFFF36
:10B93000FFFFFFFFFFFFFFFFFFFFFFFFFFFFFFFF17
:10B94000FFFFFFFFFFFFFFFFFFFFFFFFFFFFFFFF07
:10B95000FFFFFFFFFFFFFFFFFFFFFFFFFFFFFFFFF7
:10B96000FFFFFFFFFFFFFFFFFFFFFFFFFFFFFFFFE7
:10B97000FFFFFFFFFFFFFFFFFFFFFFFFFFFFFFFFD7
:10B98000FFFFFFFFFFFFFFFFFFFFFFFFFFFFFFFFC7
:10B99000FFFFFFFFFFFFFFFFFFFFFFFFFFFFFFFFB7
:10B9A000FFFFFFFFFFFFFFFFFFFFFFFFFFFFFFFFA7
:10B9B000FFFFFFFFFFFFFFFFFFFFFFFFFFFFFFFF97
:10B9C000FFFFFFFFFFFFFFFFFFFFFFFFFFFFFFFF87
:10B9D000FFFFFFFFFFFFFFFFFFFFFFFFFFFFFFFF77
:10B9E000FFFFFFFFFFFFFFFFFFFFFFFFFFFFFFFF67
:10B9F000FFFFFFFFFFFFFFFFFFFFFFFFFFFFFFFF57
:00000001FF
